:020000040800F2
:100000003810002439030008855B00902F270090EA
:1000100045030008D503009097650090000000009C
:10002000000000000000000000000000495E009099
:100030001104009000000000875B00904B5E009070
:100040005303000853030008530300085303000838
:100050005303000853030008530300085303000828
:100060005303000853030008530300085303000818
:100070005303000853030008530300085303000808
:1000800053030008530300085303000853030008F8
:1000900053030008530300085303000853030008E8
:1000A00053030008530300085303000853030008D8
:1000B00053030008530300085303000853030008C8
:1000C00053030008530300085303000853030008B8
:1000D0005303000891150008530300085303000858
:1000E00053030008530300080000000053030008F6
:1000F0005303000853030008530300085303000888
:100100005303000853030008530300085303000877
:100110005303000853030008530300085303000867
:100120005303000853030008530300085303000857
:100130005303000853030008530300085303000847
:1001400000000000000000000000000000000000AF
:100150005303000853030008530300085303000827
:100160005303000853030008530300085303000817
:100170005303000853030008530300085303000807
:1001800053030008530300085303000853030008F7
:1001900053030008530300085303000853030008E7
:1001A00053030008530300085303000853030008D7
:1001B00053030008530300085303000853030008C7
:1001C00053030008530300085303000853030008B7
:1001D00053030008530300085303000853030008A7
:1001E0005303000853030008530300085303000897
:1001F0005303000853030008530300085303000887
:100200005303000853030008530300085303000876
:100210005303000853030008530300085303000866
:1002200053030008530300085303000800000000B4
:1002300053030008530300080000000053030008A4
:100240005303000853030008530300085303000836
:100250005303000853030008530300085303000826
:100260005303000853030008530300085303000816
:100270005303000853030008530300080000000064
:1002800053030008000000005303000800000000B2
:10029000000000005303000800F002F800F03CF8F2
:1002A0000AA090E8000C82448344AAF10107DA45D1
:1002B00001D100F031F8AFF2090EBAE80F0013F0E7
:1002C000010F18BFFB1A43F001031847E4160000A2
:1002D00004170000103A24BF78C878C1FAD8520732
:1002E00024BF30C830C144BF04680C6070470000B0
:1002F0000023002400250026103A28BF78C1FBD82F
:10030000520728BF30C148BF0B6070471FB501F0CE
:1003100041FB1FBD10B510BD00F0AAF81146FFF754
:10032000F5FF01F0A5F900F0C8F803B4FFF7F2FFFC
:1003300003BC01F05FF90000094880470948004705
:10034000FEE7FEE7FEE7FEE7FEE7FEE7FEE7FEE785
:10035000FEE7FEE704480549054A064B70470000E2
:100360000D150008990200083804002438100024F4
:100370003806002438060024704753EA020C00F0C7
:1003800069802DE9F04B4FF00006002B1FBFB3FA38
:1003900083F503FA05F424FA05F65E4012BF16430E
:1003A000B2FA82F502FA05F4C5F120051EBF22FA61
:1003B00005FC44EA0C04203556EA044C4FEA144488
:1003C00018BF641C4FF000084FF00009904271EB19
:1003D000030C39D3002919BFB1FA81F701FA07F6E6
:1003E000B0FA80F700FA07F6C7F120071EBF20FA1F
:1003F00007FC46EA0C062037B6FBF4FCA7EB050722
:10040000103F07F01F0BCBF120060CFA0BFB2CFA68
:1004100006F644BFB3460026202FA4BF5E464FF029
:10042000000B5BEA060C08BF4FF0010B19EB0B0940
:10043000ABFB027C48EB0608C01B06FB02CC0BFBA7
:1004400003CC71EB0C01C1E70B460246414648461E
:10045000BDE8F08B13B54FF000004FF00001AFF393
:100460000080BDE81C407047704770477047704778
:10047000754600F02BF8AE4605006946534620F05D
:100480000700854618B020B5FFF764FFBDE820409F
:100490004FF000064FF000074FF000084FF0000B40
:1004A00021F00701AC46ACE8C009ACE8C009ACE8F3
:1004B000C009ACE8C0098D46704710B50446AFF3DB
:1004C00000802046BDE81040FFF72FBF004870476E
:1004D000D403002441F2D56CC9F2000C604742F20B
:1004E0009D4CC9F2000C604742F2914CC9F2000CDD
:1004F000604742F2876CC9F2000C604745F2ED3C60
:10050000C9F2000C604742F2317CC9F2000C60472E
:1005100045F6695CC9F2000C604742F6C12CC9F28D
:10052000000C604745F6353CC9F2000C604740F2CC
:10053000D93CC9F2000C604745F2BD2CC9F2000C51
:10054000604741F21D3CC9F2000C604742F2B17CA9
:10055000C9F2000C604741F29D2CC9F2000C6047C3
:1005600045F2113CC9F2000C604740F2E50CC9F2BB
:10057000000C604740F2676CC9F2000C604742F221
:100580001D6CC9F2000C6047F0B5BFF34F8FBFF38D
:100590006F8F1D4900200860BFF34F8FBFF36F8F2F
:1005A0001A4C216841F400312160BFF34F8FBFF333
:1005B0006F8F164970310860BFF34F8F081F0068B6
:1005C00043F6FF75104E1036C0F34E31C0F3C90329
:1005D00005EA4112184642EA80773760401EFAD297
:1005E000491EF5D2BFF34F8F206840F48030206061
:1005F000BFF34F8FBFF36F8F03484C30016841F05A
:1006000004010160F0BD000050EF00E014ED00E0D7
:1006100070B5044600F018F90546601C02D0044885
:100620000078044400F010F9401BA042FAD370BDDA
:10063000140000240248016841F001010160704784
:10064000200400582DE9F84F6C4C00224FF0B04ABE
:100650004FF0010B4FF0030E4FF00F090B680BFA30
:1006600002F73B40BB4270D14D68022D01D0122DE4
:1006700012D1D50800EB850CDCF820605507ED0E93
:1006800009FA05F826EA0806D1F8108008FA05F8F4
:1006900048EA0608CCF82080D0F80080560091F88F
:1006A00004C00EFA06F50CF0030C28EA05080CFA53
:1006B00006FC4CEA080CC0F800C0D1F804C0BCF13C
:1006C000010F08D0BCF1020F05D0BCF1110F02D010
:1006D000BCF1120F16D1D0F808C0D1F80C802CEA6A
:1006E000050C08FA06F848EA0C08C0F80880D0F8AB
:1006F00004C02CEA070C0F79C7F30017974047EAAC
:100700000C074760C768AF438D68B5403D43C5607F
:100710004D68ED006BD53A4D2E6846F002062E600E
:100720002D6822F0030606F1B04605F0020500959B
:10073000D6F808C495072F0F09FA07F52CEA050C1F
:10074000304DA84202D100252EE050E02E4DA842A7
:1007500001D1012528E02D4DA84201D1022523E039
:100760002B4DA84201D103251EE02A4DA84201D1FC
:10077000042519E0284DA84201D1052514E0274D94
:10078000A84201D106250FE0254DA84201D1072539
:100790000AE0244DA84201D1082505E0224DA842D7
:1007A00001D1092500E00A25BD4045EA0C05C6F83F
:1007B000085425684E689D43F60300D51D43256007
:1007C00065684E689D43B60300D51D436560DAF841
:1007D000005056464F689D43FF0200D51D433560CB
:1007E00075684F689D43BF0200D51D437560521C5C
:1007F000102AFFF433AFBDE8F88F000080000058E6
:10080000F44402580000025800040258000802583C
:10081000000C025800100258001402580018025828
:10082000001C0258002002580024025800690840A9
:1008300000D00120704742694A40426170470AB1C6
:10084000018370474183704701488068704700000A
:1008500014000024024881680278114481607047C6
:1008600014000024032010B500F0A2F80F2000F0BF
:1008700007F808B1012010BD00F06CF8002010BD91
:1008800070B50D4D04464FF47A712878B1FBF0F045
:100890000A490968B1FBF0F000F0A4FC48B9102C3B
:1008A00007D200222146501E00F062F800206C6042
:1008B00070BD012070BD0000140000240000002461
:1008C000134A41781160111D03780A1DE3B1436892
:1008D0000B60017BC37A090741EA0361837A41EA2D
:1008E000C341437B41EA8341837B41EA4341C37B6C
:1008F00041EA0341437A41EA0321037A007841EA5D
:100900004301014311607047002008601060704788
:1009100098ED00E0BFF35F8F0448016821F4803157
:1009200001600249002070310860704724ED00E04A
:10093000074940F00100086005487038016841F43B
:1009400080310160BFF34F8FBFF36F8F704700009E
:1009500094ED00E07047002809DB012100F01F0240
:1009600091404009800000F1E020C0F8001170477C
:100970000E4BF0B41B68C3F30223C3F10704042C2D
:1009800000D904241D1D072D01D2002300E0DB1E29
:10099000012606FA04F56D1E0D409D409E40761E10
:1009A000164045EA0601F0BC00F014BE0CED00E074
:1009B000064A00F0070110684FF6FF03184040EAAE
:1009C0000120034908431060704700000CED00E06F
:1009D0000000FA052DE9F047DFF8BC9104460E4609
:1009E000D9F8000000F00700B0420CD2D9F800108E
:1009F00021F007013143C9F80010D9F8000000F0D8
:100A00000700B0427ED12078DFF89081800707D5BB
:100A1000D8F80010E26821F00F011143C8F8001067
:100A20002078C00762D0D8F80010A26821F4706165
:100A30001143C8F8001059496068183902281CD0C1
:100A400003281DD0096801281DD04907002960DA54
:100A5000524F083F396821F0070101433960FFF721
:100A6000F3FE0546606841F28831022813D003285E
:100A70001ED001288A4627D034E009688903E5E7BB
:100A800009688901E2E7C905E0E7FFF7DDFE411BE0
:100A9000514501D923E08A463868C0F3C2000228D4
:100AA000F3D123E0FFF7D0FE411B514501D916E0F9
:100AB0008A463868C0F3C2000328F3D116E0FFF776
:100AC000C3FE411B51450AD83868C0F3C200012853
:100AD000F5D10BE0FFF7B8FE411B514502D90320C9
:100AE000BDE8F087386810F0380FF3D1D9F800105E
:100AF000484601F00701B1420DD9016821F0070114
:100B0000314300E005E00160006800F00700B042FA
:100B100001D00120E4E72078400707D5D8F800107D
:100B2000226921F070011143C8F8001020780107F4
:100B30001B4805D50168626921F07001114301600D
:100B40002178C90605D50168A26921F4E061114345
:100B500001602078800607D51149091D0868E269FF
:100B600020F070001043086000F066F8D8F800101C
:100B70004FF4807292FAA2F201F47061B2FA82F23A
:100B8000D140084A515CC840074908600F20FFF770
:100B900077FE0020A4E7000000200052184402580D
:100BA0001C4402589E1900080000002410B5FFF7ED
:100BB00091FC08490968012292FAA2F201F00F01A2
:100BC000B2FA82F2D140044A515CC840034908603D
:100BD00010BD0000184402589E19000804000024AB
:100BE00010B5FFF7E3FF07490968102292FAA2F255
:100BF00001F07001B2FA82F2D140034A515CC84060
:100C000010BD00001C4402589E19000810B5FFF7E3
:100C1000CDFF074909684FF4807292FAA2F201F4FD
:100C2000E061B2FA82F2D140024A515CC84010BD84
:100C30001C4402589E1900083548F0B50068364D2E
:100C400010F03801334809D00411082904D0334E7C
:100C500010290BD018290BD02046F0BD2968890631
:100C6000FBD52968C1F3C101C840F0BD3046F0BDD5
:100C7000274918310A68096812F00302284BC1F3AA
:100C800005111B68274F03F001033F68DFED260ABB
:100C9000B7EE001AC7F3CC0717FB03F300EE103AC8
:100CA000224BB8EE400A06D0012A01D0022A2BD0EE
:100CB000B4FBF1F008E02A68920603D52A68C2F373
:100CC000C102D040B0FBF1F001EE900A1868B8EE16
:100CD000612AC0F3080001EE900A1868F8EE611A64
:100CE00040EE201A31EE810A22EE000AC0F34620BF
:100CF000401C00EE900AF8EE600A80EE201ABCEE6E
:100D0000C10A10EE100AF0BDB6FBF1F0DCE70000FE
:100D1000104402580090D0030044025840787D01EE
:100D20002C44025834440258000000393044025820
:100D30002DE9F05F04460078DFF8FC8341F2883942
:100D4000DFF8F8A3FE4DC0074ED0D8F8001040469B
:100D5000C1F3C20102291AD00068C0F3C2000328FF
:100D600005D1DAF8000000F0030002280FD0606817
:100D7000B0F5803F12D010B1B0F5A02F19D028687F
:100D800020F480302860286820F4802009E028685A
:100D9000800329D56068002874D025E0286840F4D5
:100DA00080302860606890B1FFF74EFD06464F46E0
:100DB00009E0286840F480202860EFE7FFF744FD51
:100DC000801BB8427DD828688003F7D50CE0FFF778
:100DD0003BFD06464F4604E0FFF736FD801BB84258
:100DE000F0D828688003F7D42078D64F80075AD5EA
:100DF000D8F8001040464FF47C3B11F0380F13D068
:100E00000068C0F3C200032803D1DAF800008007AD
:100E10000AD0E068A8B3296821F0190101432960CC
:100E2000FFF712FD06461DE02868400702D5E0687E
:100E30000028B1D02868E16820F019000843286034
:100E4000FFF702FD064604E0FFF7FEFC801B0228C8
:100E5000B8D828684007F7D507E0FFF7F5FC801BF6
:100E60000228AFD828684007F7D538689BFAABF25C
:100E700020F47C312069B2FA82F29040014339605B
:100E800011E000E0AEE0286820F001002860FFF7E4
:100E9000DBFC064604E0FFF7D7FC801B022891D854
:100EA00028684007F7D42078C00655D5D8F8001038
:100EB00040464FF0F84BC1F3C201012917D000683A
:100EC00000E0EDE0C0F3C200032805D1DAF800002D
:100ED00000F0030001280AD0E069002828682CD01F
:100EE00040F080002860FFF7AFFC064616E0286857
:100EF000C00502D5E069802874D138689BFAABF24E
:100F000020F0F841206AB2FA82F290400143396041
:100F100022E0FFF799FC801B022899D82868C005B9
:100F2000F7D538689BFAABF2216AB2FA82F220F068
:100F3000F8409140084338600EE020F080002860BF
:100F4000FFF782FC064604E0FFF77EFC801B0228C8
:100F500087D82868C005F7D42078000724D5774FB4
:100F600060694C37002838680FD040F001003860C5
:100F7000FFF76AFC064604E0FFF766FC801B0228C8
:100F80008DD838688007F7D50EE020F00100386072
:100F9000FFF75AFC064604E0FFF756FC801B0228C8
:100FA0007ED838688007F7D42078800623D5A069DA
:100FB000002828680FD040F480502860FFF744FCD8
:100FC000064604E0FFF740FC801B022868D828682A
:100FD0008004F7D50FE020F480502860FFF734FC40
:100FE000064605E0D6E0FFF72FFC801B022857D805
:100FF00028688004F7D42078400744D5524F3868D9
:1010000040F480703860FFF71FFC064604E0FFF7ED
:101010001BFC801B642843D83868C005F7D5474FB0
:10102000A068483701280AD008B1052811D03868CF
:1010300020F001003860386820F0040002E03868D1
:1010400040F001003860A06888B1FFF7FDFB06465C
:1010500009E0386840F004003860F0E7FFF7F4FB7F
:10106000811B49451CD838688007F7D50BE0FFF78E
:10107000EBFB064604E0FFF7E7FB811B49450FD871
:1010800038688007F7D4606AF0B3D8F80010C1F36D
:10109000C20103297ED00228286820F0807000E079
:1010A00079E0286003D0FFF7CFFB044687E0FFF725
:1010B000CBFB064604E0FFF7C7FB801B02287BD86A
:1010C00028688001F7D4DAF8001040F2F332914337
:1010D000E26A41EA0211A26A1143CAF8001094F8C8
:1010E00034004FF4FE02218E4002491EA0F500702C
:1010F00080B2C1F308010843218F491E02EA014171
:10110000084394F83C1000E05CE0491E120202EA39
:10111000016108430949083108600B1D19684FF641
:10112000F872A06C914392FAA2F2B2FA82F2904065
:1011300001431960014809E010440258284402584C
:10114000004402580444025800480258001D016837
:10115000226C21F00C01114301600168626C21F0E6
:10116000020111430160016841F4803101600168AE
:1011700041F400310160016841F48021016001689F
:1011800041F001010160286840F080702860FFF79D
:101190005BFB01E018E00FE0044604E0FFF754FBBE
:1011A000001B022808D828688001F7D50AE0FFF75D
:1011B0004BFB001B022802D90320BDE8F09F2868E2
:1011C0008001F4D40020F8E70120F6E74FF0E02199
:1011D0000428086903D020F004000861704740F03B
:1011E0000400FAE7401EB0F1807F10B501D3012062
:1011F00010BD4FF0E02460610F21601700F0EAF9A4
:101200000020A06107202061002010BD10B50068FB
:1012100086B01B49884230D11A48016841F001016B
:101220000160006800F00100059016481030016868
:1012300041F01001016000680121134C00F0100022
:1012400005904FF4007000900220CDE90101039059
:101250000720694604902046FFF7F4F94FF48061B7
:10126000204600916946FFF7EDF92520FFF773FB53
:10127000032225201146FFF77BFB06B010BD0000BE
:1012800000100140E04402580000025830B50068E8
:10129000114988420CD1114A5088010408D41146E2
:1012A0004FF000034404097806D50A2901D0538081
:1012B00030BD40F400400DE00D2909D0084DC0F3C9
:1012C0000D04401C80B2C72829555080EFD830BD8E
:1012D00040F48040508030BD001001400C000024DC
:1012E0003400002454482DE9F041524C86B0016886
:1012F00041F002010160016841F0200101604E48A7
:101300000C38016841F480410160402000900220C7
:1013100001900320DFF82481002569460A270497FD
:10132000CDE902504046FFF78DF9042069460926B1
:10133000049600904046FFF785F90496C020404E81
:10134000694600903046FFF77DF94FF440706946DA
:10135000049700903046FFF775F937486438016804
:1013600041F480410160016821F48041016031480D
:10137000203881688906FCD43249016032494160D5
:10138000016841F00101016081688906FCD44FF4D5
:101390009C71416181688907FCD5C16841F00201F7
:1013A000C16081688906FCD44FF483714161816812
:1013B0008907FCD5C16841F00201C16081688906D6
:1013C000FCD422494161056181684907FCD530217F
:1013D0002170016841F00401016081688907FCD532
:1013E000C16841F00201C16081688906FCD481684E
:1013F0008906FCD4C561164941611648016821F48B
:1014000080310160134970310A6822F001020A60DC
:101410000A1D156082060F4B78331A601B1D0E4A99
:101420001A6005220A60016841F48031016006B04B
:10143000BDE8F08120500052E044025800040258F8
:10144000001402581003000101041600C003000339
:10145000EBEF180F24ED00E02D00030370B5294CCD
:101460009CB0256825F004052560264C00260C3428
:10147000256845F440452560256805F440451B95E1
:101480002568AD04FCD5012400940CAD039624041A
:10149000019402240994CDE90A410796082485E8BD
:1014A0000D00CDE910466846FFF742FC98B9FFF7FA
:1014B00019FF3F2013900320CDE9140640200101BD
:1014C000CDE91640CDE9180150201A90022113A849
:1014D000FFF780FA10B101201CB070BD0A48016806
:1014E00041F0800101600848F430016841F00201D8
:1014F0000160006800F002001B90FFF79BF80020DD
:10150000EAE700000C480258004402581C480168F1
:1015100041F4700101601B49086840F00100086057
:10152000184A0020103210600A68174B1A400A60EF
:10153000144A18321060121D1060121D1060114AFA
:1015400028321060121D1060121D1060121D1060F4
:10155000121D1060121D1060121D1060121D10600F
:101560000A6822F480220A6006496031086001207E
:101570000649C1F80801C006014980390860704772
:1015800088ED00E0004402587FEDF6EA008000514B
:1015900070B50D4D00240D48FEF7A1FF02E0641C5C
:1015A000AC4204D80948FEF79FFF2028F7D1002459
:1015B00002E0641CAC4206D8054901220348FEF74C
:1015C00098FF0028F5D170BDFFFF0100FC0000244A
:1015D0000C0000240907090E002804DB00F1E020BC
:1015E00080F80014704700F00F0000F1E02080F850
:1015F000141D70477047000010B504460420FFF723
:10160000E5FD0148046010BD0800002470B5002409
:1016100005464FF47A7603E0304600F005F8641C86
:10162000AC42F9D370BD000070B54FF0E025002149
:101630006C69094AAB6912685043AA699A42FCD0A6
:1016400002D2A3EB020302E0A4EB020633441944E6
:1016500013468142F1D370BD080000240349CA69D2
:101660005206FCD5C2B20A85704700000010014046
:1016700000272DED028BB0B03C46FEF785FFFFF74B
:10168000F1F8042302220521A020FFF7E7FE4FF422
:10169000C870FFF7B1FF4FF4E13000F05FF9FEF7DB
:1016A0002DFFFEF730FFFEF733FFFEF736FFFEF7A4
:1016B00039FFFEF73CFF834E4FF478401025C822D7
:1016C0002B463221306080A0CDE900501E20FEF76D
:1016D00033FF81A01023C822CDE9005046211E20EF
:1016E000FEF72AFF7FA01023C822CDE900505A211F
:1016F0001E20FEF721FF7FA01023C822CDE9005055
:101700006E211E20FEF718FF7DA01023C822CDE910
:10171000005082211E20FEF70FFF1F2030607CA0AA
:101720001023C822CDE9005096211E20FEF704FFA9
:101730007AA01023C822CDE90050AA211E20FEF76E
:10174000FBFE7AA01023C822CDE90050BE211E2046
:10175000FEF7F2FE002379481A461946FEF7F1FE1D
:101760007F1C0020FFB2FEF7F1FE0428064602D0DF
:10177000022E05D010E0B4F57A6F07D2C83402E02B
:10178000C82C02D9C83CA4B200E000246B48002257
:1017900023461146FEF7D5FE0A2F03D0022E01D0B4
:1017A000042E7DD165480021FEF7D5FE002687B2C4
:1017B00004233A4696215E20CDE90056FEF7D0FE7E
:1017C00000EE107AB8EE400B9FED5D1B0123AA21BD
:1017D00020EE010BCDE90056B7EEC08BBCEEC80A77
:1017E00010EE100A10EE102A87B25E20FEF7B8FE47
:1017F00000EE107AB8EE400A38EE400ADFED528A69
:101800004FF08008032320EE280AAA216E20CDE99C
:101810000058BCEEC00A10EE102AFEF7A1FE4B499C
:10182000542217A8FEF7A1FE4848416D2C91816D06
:101830002D91C16D006E5422CDE92E100A21132086
:10184000CDE915011BA96846FEF78FFE0DF15C0C72
:101850009CE80F00FEF78EFE00EE100A9FED3C1B89
:101860000123B8EE400BBE21CDE9005620EE010B5E
:10187000B7EEC08BBCEEC80A10EE100A10EE102AAC
:1018800087B25E20FEF76CFE00EE107A0323B8EEFE
:10189000400A38EE400A20EE280ABCEEC00A00E0FA
:1018A0000CE0BE216E2010EE102ACDE90058FEF7A4
:1018B00057FE29480221FEF7BEFF00270A20FFF746
:1018C000A5FE4DE72400002441706F6C6C6F20531F
:1018D000544D33324837000044414320544553545B
:1018E0000000000041544F4D40414C49454E544585
:1018F0004B000000323031372F382F3134000000D8
:10190000574B5F55503A2B20204B4559313A2D000B
:101910004441432056414C3A0000000044414320DA
:10192000564F4C3A302E3030305600004144432060
:10193000564F4C3A302E3030305600009C03002475
:101940006666666666664A3F00007A44D4020024F2
:101950006666666666660A3F000402580B490A4AD4
:1019600010B5C1E9002000208860C8600861886166
:101970000C2048610846FEF702FEBDE8104004490D
:1019800001220248FEF7B5BD00100140FC00002412
:101990000C0000244FF04070E1EE100A7047000088
:1019A0000000010203040102030406070809000005
:1019B000D01900080000002434000000D402000800
:1019C000041A00083400002404100000F00200088B
:1019D0000090D0030090D003000000000000000041
:1019E00000000000010000001000000000000000E6
:1019F00001000000000000FFFFFFFFFF00000000EB
:041A000000000000E2
:0200000490006A
:10000000782900F043800020704700000FB40449B5
:1000100010B503AA029800F0F1F810BC5DF814FBCB
:10002000100000242DE9F0410E4604460020206215
:100030002046E168884730B3252805D0D4E901215E
:100040009047206A401CF2E7E16820460027884775
:10005000050018D0A5F14100192802D820354FF429
:1000600000673246294620462760FFF7C9FF40B1A6
:10007000012804D0F61D26F007060836D8E7361DFD
:10008000D6E72846DAE7206ABDE8F08170B5044675
:100090000D4621461068AFF300802188090502D57E
:1000A0000F4A7A4402E00E4A7A440E32002104F1EB
:1000B000240305E000F00F060009965D5E54491C1C
:1000C0000028F7D120780023000704D5702D02D036
:1000D00009B1022311322046BDE8704000F034B867
:1000E0004AAC000010B5203AC0F00B80B1E81850BF
:1000F000203AA0E81850B1E81850A0E81850BFF412
:10010000F5AF5FEA027C24BFB1E81850A0E81850B0
:1001100044BF18C918C0BDE810405FEA827C24BF04
:1001200051F8043B40F8043B08BF7047D20728BF92
:1001300031F8023B48BF11F8012B28BF20F8023BE1
:1001400048BF00F8012B70472DE9F0470D4699464E
:100150009246044600F124080168880604D5E06947
:1001600021F01001216000E00120A84201DD471BC1
:1001700000E00027A1697A1902EB0900081AA061C2
:100180002078C00602D42046AFF30080002608E0A5
:10019000D4E901211AF806009047206A401C761C19
:1001A00020624E45F4DB2078C0060AD52046AFF326
:1001B000008006E0D4E9012130209047206A401CED
:1001C0002062381EA7F10107F4DC07E0D4E9012121
:1001D00018F805009047206A401C2062281EA5F1EF
:1001E0000105F3DC2046AFF300802078000602D53D
:1001F0000220BDE8F0870120FBE70000074B70B547
:100200000D467B4400F011F80446284600F020F823
:1002100010B14FF0FF3070BD204670BD571400780C
:1002200001694A1C02610878704700B58FB0CDE9BA
:1002300001310021059105497944CDE903101146AA
:100240006846FFF7EFFE0FB000BD0000E5FFFFFFBF
:10025000007B00F08000704740F6490CC0F6000CAF
:10026000604741F20D6CC0F6000C604740F2456CEF
:10027000C0F6000C604740F2116CC0F6000C6047FD
:1002800040F6394CC0F6000C604740F6AD3CC0F675
:10029000000C604741F20D2CC0F6000C604740F6A0
:1002A0002D0CC0F6000C604741F2296CC0F6000C22
:1002B000604740F63F0CC0F6000C604740F6151C46
:1002C000C0F6000C604740F6C10CC0F6000C604759
:1002D00040F6311CC0F6000C604740F6550CC0F6E5
:1002E000000C604741F28D2CC0F6000C604740F2D4
:1002F0007B3CC0F6000C604740F6E13CC0F6000CC9
:10030000604740F60D4CC0F6000C604770B50446DF
:100310000068816801F00301012925D10168C9073E
:1003200022D0816801F00D0101290FD1816841F0CF
:1003300002018160216803200860FFF78DFF0546F8
:100340000EE0FFF789FF401B022809D9606D40F0DD
:1003500010006065A06D40F00100A065012070BD37
:1003600020688068C007ECD1002070BD70B50446DD
:100370000068816801F00301012902D10168C90701
:1003800023D18168124A114210D1816841F00101E4
:100390008160FFF761FF054612E0816841F00101CD
:1003A0008160FFF759FF401B022809D9606D40F0BA
:1003B00010006065A06D40F00100A065012070BDD7
:1003C00020680168C943C907E7D1002070BD00005B
:1003D0003F000080FEE700000C490B4810B50860A4
:1003E000084600F061FF09480021002214304160F6
:1003F000022181600146143800F0CAFEBDE81040B9
:100400000248002100F097BF007400409C030024C4
:100410007047000070B5B3F5804F05D06FF07041A4
:1004200040F82210002070BD50F82230084C2340C4
:10043000D1E900458E8944EA05148D6889692D0249
:1004400045EA06452C430C431C4340F82240E9E7AB
:100450000000F0CFF0B50C6850F824501A4A15404F
:10046000D1E90123D1E903671A433E4332434E6980
:1004700032438E693243CE6932430E6A32434E6A4A
:1004800032438E6A3243CE6A32430E6B32438E6BF6
:1004900032434E6B32432A43082B01D142F04002D3
:1004A00040F824200A6BB2F5801F05D10A684AB1D2
:1004B000026842F4801202600A681AB10268496B4D
:1004C0000A4302600020F0BD8004C0FF00EB8202FE
:1004D000F0B553688E8903F04044D1E9003543EA12
:1004E00005138D682D0245EA06450E8A2B430D4DF6
:1004F00005EB065633430E7D6F0107EB066633436B
:100500008E693343234353600268D20207D54268A1
:10051000098A22F4700205EB015111434160002069
:10052000F0BD00000000F0FF30B5D1E901230D68F7
:100530001A43D1E9033423431A434B691A438B69A5
:100540001A43D1E90734496A012D056807D01A43D7
:1005500022430A436FF30E052A4302600AE025F4A2
:10056000F845234329430B43416803606FF30E01B1
:100570000A434260002030BD426942EA41014161C4
:100580000020704718B5D1E900236FF01F041A430B
:100590008B68C96804EB431343EA41210A43009284
:1005A0000261002018BD0000F0B5D1E900346FF001
:1005B0000F055B1E2E0105EB041423438C682F03EB
:1005C0004FEA054C0D8A06EB04248E8A2343CC683F
:1005D000097E4FF07F4E012A07EB05450CEB0656CE
:1005E0000EEB01610CD082683F1107EB043423430A
:1005F0002B4333430B4302F07042134383600FE0FD
:100600008768084A17402203C468A2F58052324323
:100610003A4382602B430B4304F070442343C3608E
:100620000020F0BDFF0F0FFF0FB400B587B0694683
:100630002198009001200190072002900020039053
:100640000490059008A800F091F808A800F028FD93
:100650000A2108A800F088FC08A800F01BFB07B0DE
:1006600080B25DF814FB0FB42DE9F041B0B0002565
:100670000DF168082C46DDE94F761EE0542236A9BC
:1006800016A8FFF72FFD4B982B904C982C904D9867
:100690004E9954221597CDE92D0141466846FFF742
:1006A00021FD0DF1580C9CE80F00FFF7BDFF05443C
:1006B0000520FFF7D6FD641CE4B2B442DED3B5FBDF
:1006C000F6F030B0BDE8F00180B25DF814FB2DE922
:1006D000F041044690F850000025164601280F46C8
:1006E0000CD0012084F850002046FFF70FFE0100D7
:1006F000606D2A4605D040F0100031E00220BDE8D0
:10070000F08120F4885040F0020060652068836822
:1007100023F08043334383602068836823F480336D
:100720003B4383602068836843F000438360206814
:100730004FF47A460CE06D1CB54209D3606D20F091
:10074000020040F010006065012084F85020D6E7D8
:100750008368002BEFDB606D20F0020040F00100A9
:100760006065084684F85020C9E700002DE9F84F7D
:100770000023FC4C4FF0804E9B46009390F8502095
:10078000012A28D0012580F8505002689668760723
:100790007ED4D669AA460F78BD402E43D6614A68FA
:1007A0001F254FF4F868052A18D20668376B98FAA7
:1007B000A8FCBCFA8CFC02FB0CFC05FA0CF598FAC0
:1007C000A8FCAF430D68BCFA8CFC02FB0CF2954010
:1007D0002F43376349E00220BDE8F88F0A2A16D27A
:1007E0000668776B98FAA8FC521FBCFA8CFC02FBD7
:1007F0000CFC05FA0CF598FAA8FCAF430D68BCFA9E
:100800008CFC02FB0CF295402F4377632DE00668C9
:100810000F2A15D2B76B98FAA8FC0A3ABCFA8CFCDE
:1008200002FB0CFC05FA0CF598FAA8FCAF430D6826
:10083000BCFA8CFC02FB0CF295402F43B76314E02A
:10084000F76B98FAA8FC0F3ABCFA8CFC02FB0CFC84
:1008500005FA0CF598FAA8FCAF430D68BCFA8CFCBD
:1008600002FB0CF295402F43F763026895684FF046
:1008700038064FF0070915F00C0F7DD10D680A2DD1
:100880001BD3976996FAA6FC0A3DBCFA8CFC00E0E3
:10089000C9E105FB0CF809FA08FC96FAA6F827EA64
:1008A0000C07D1F808C0B8FA88F805FB08F50CFA6F
:1008B00005FC47EA0C07976117E0576996FAA6FC12
:1008C000BCFA8CFC05FB0CF809FA08FC96FAA6F8B1
:1008D00027EA0C07D1F808C0B8FA88F805FB08F534
:1008E0000CFA05FC47EA0C07576102684D69D768A6
:1008F0004FF0F84CC7F382077F00BD400F69012F0E
:100900004AD0022F6AD0032F7DD0042F7CD0156EE1
:100910009CFAACF805F0F8470D68B8FA88F805FAC3
:1009200008F5AF4203D1156E25F000451566026843
:10093000556E9CFAACF805F0F8470D68B8FA88F8DF
:1009400005FA08F5AF4203D1556E25F0004555660E
:100950000268956E9CFAACF80F68B8FA88F805F052
:10096000F84507FA08F7BD4203D1956E25F000451A
:1009700095660268D56E00E02FE09CFAACFC05F0AD
:10098000F8470D68BCFA8CFC05FA0CF5AF4224D18F
:10099000D56E25F0004589E0176E9CFAACFC07F097
:1009A00000480F68BCFA8CFC07FA0CF72F4348EAA2
:1009B0000708C2F86080026815690F7E25F400659B
:1009C0003D4315614A7E002A0268156E02D045F04B
:1009D000004501E025F00045156668E0576E9CFA79
:1009E000ACFC07F000480F68BCFA8CFC07FA0CF767
:1009F0002F4348EA0708C2F86480026815690F7E31
:100A000025F4805501E00FE031E045EA4705156126
:100A10004A7E002A0268556E02D045F0004501E08A
:100A200025F00045556642E0976E9CFAACFC07F055
:100A300000480F68BCFA8CFC07FA0CF72F4348EA11
:100A40000708C2F86880026815690F7E25F4005512
:100A500045EA870515614A7E002A0268956E02D034
:100A600045F0004501E025F0004595661FE0D76E92
:100A70009CFAACFC07F000480F68BCFA8CFC07FA43
:100A80000CF72F4348EA0708C2F86C800268156922
:100A90000F7E25F4804545EAC70515614A7E002A88
:100AA00002683FF475AFD56E45F00045D566026823
:100AB000956805F00305012D02D11568ED0761D198
:100AC000CD68754507D052F8C06F0F780AFA07F560
:100AD000AE4316603CE052F8C07F91F800C00AFABD
:100AE0000CF52F4317600A680568092A18D3AF6907
:100AF00096FAA6FC093ABCFA8CFC96FAA6F602FB1A
:100B00000CF8B6FA86F609FA08FC724327EA0C07D5
:100B1000D1F808C00CFA02FC47EA0C07AF6117E0F5
:100B20006F6996FAA6FC521CBCFA8CFC96FAA6F6E3
:100B300002FB0CF8B6FA86F609FA08FC724327EABB
:100B40000C07D1F808C00CFA02FC47EA0C076F61E9
:100B5000054E0568054FB54201D0BD420AD1044A91
:100B600009E000000060025800200240002102401D
:100B700000230240444A0968122904D0112907D0F1
:100B800013290AD054E0D2F808C04FEA0C2C08E030
:100B9000D2F808C04FEACC1C03E0D2F808C04FEAF4
:100BA0004C2CBCF1000F43DBD5F808C00CF0030C53
:100BB000BCF1010F04D1D5F800C05FEACC7C32D182
:100BC000B54210D1D6F8087107F00307012F03D101
:100BD000D6F80061F60726D1A66806F00306012EB6
:100BE0002AD126681DE0BD42B76807F003070BD184
:100BF000012F02D13768FF0715D1A76807F0030757
:100C0000012F06D1276802E0012F02D13768FF07C4
:100C100009D1D6F8087107F00307012F0CD1D6F8D7
:100C20000061F60708D0416D41F0200141650123C4
:100C300080F850B01846CFE512290AD011291CD0EF
:100C40001329F5D1A542F3D1916841F48001916057
:100C5000EEE7A542ECD1916841F4000191600B49A7
:100C60000B4A0968B1FBF2F1C1EB0111C90000E0C8
:100C7000491E00910029FBD1DAE7A542D8D191683D
:100C800041F08071E3E70000006302580000002497
:100C900080841E000068006C70470000F8B54FF0BB
:100CA000000504002E46009502D0606D10B107E0EB
:100CB0000120F8BD204600F021F9A66584F85060B7
:100CC00020688168890003D5816821F00051816026
:100CD00020688168C90010D4816841F0805181602A
:100CE0007D487E490068B0FBF1F000EB80004000D9
:100CF00000E0401E00900028FBD120688168C900F8
:100D000008D4616D41F010016165A16D41F00101F0
:100D1000A1650125616DC9067ED481684907FBD4B0
:100D2000616D41F0020161656D4A6E4E904201D0E5
:100D3000B04201D16C4900E06C49836803F00303C1
:100D4000012B02D10368DB0739D1694B904210D1E6
:100D5000D2F8080100F00300012803D1D2F8000105
:100D6000C0072CD1986800F00300012821D1186831
:100D70001DE0B042906800F003000BD1012802D1C1
:100D80001068C0071BD1986800F00300012806D145
:100D9000186802E0012802D11068C0070FD1D2F80C
:100DA000080100F00300012803D1D2F80001C007B8
:100DB00005D18868626820F47C1010438860A168BF
:100DC0004FF48033206B627D93FAA3F308434FF412
:100DD0000051B3FA83F391FAA1F1B1FA81F18A409B
:100DE000217F01FA03F31A431043012909D14FF47B
:100DF0006022216A92FAA2F2491EB2FA82F291406E
:100E00000843616A012903D0A26A0AB11143084369
:100E10002168CA68374B00E056E01A400243CA60B6
:100E20002068816811F00C0F28D14FF48042217D99
:100E300092FAA2F2B2FA82F29140E26A1143C268D7
:100E400044F203039A430A43C26094F8390001282C
:100E50001CD02068016921F001010161206801694D
:100E6000626B21F070411143016194F83800012850
:100E7000206881681AD021F480718160E0680128BF
:100E80002068016B21F00F0113D015E0D4E9101098
:100E9000A28F01230143A06C03EB024210430143E4
:100EA00020680269144B1A401143D6E741F480715F
:100EB000E3E7A269521E11430163606D20F0020056
:100EC00040F00100606504E0606D40F01000606576
:100ED00001252846F8BD00000000002480841E0083
:100EE000002002400021024000230240006302581B
:100EF0000060025803C0F0FF1EF800FC184800B55F
:100F0000B5B0016841F020010160006800F02000E8
:100F1000349013480830016841F080710160016825
:100F200001F080713491016841F0010101600068B5
:100F300000F0010034904FF40020009080102890C1
:100F4000684600F0F3FC20202F9003203090002012
:100F5000319004482FA9FFF789F935B000BD000092
:100F6000D8440258000002582DE9F04704460069B1
:100F7000DFF81C91012608280F4622D02068494638
:100F8000884202D0434A90421DD1D1F80823D206AC
:100F900019D0D1F8082302F01F02052A13D0D1F886
:100FA000081301F01F0109290DD03B488168C1F3E6
:100FB000813102290AD08068C0F38130032805D02E
:100FC0000BE008250AE0C068C00706D0606D40F05D
:100FD000200060650120BDE8F0870425FFF73CF99B
:100FE000804611E0781C0FD02FB1FFF735F9A0EB48
:100FF0000800B84208D9606D40F004006065002028
:1010000084F850000320E6E7206800682842E9D011
:1010100020680168090700D400264946884224D088
:101020001E4A904221D0D1F80823D2061DD0D1F813
:10103000082302F01F02052A17D0D1F8082302F076
:101040001F02092A11D0C968082D10D04A0401D402
:1010500004220260606D40F400706065B6B12068E3
:10106000C06810F4406F04D010E0C168ECE70822BB
:10107000EFE788040AD4606D20F480706065606DCD
:10108000C00403D4606D40F0010060650020A2E759
:10109000002002400021024000230240006002586C
:1010A00070B5044600688068400767D494F8500023
:1010B00001280AD0012084F850002046FFF756F995
:1010C00001004FF0000202D045E0022070BD606DCB
:1010D000C00404D5A06D20F00600A06500E0A26564
:1010E000606D40F60163984340F480706065254B65
:1010F0002068984206D0244DA84203D0D3F8085364
:10110000ED0603D1656D25F4801565651C25056028
:101110002068984222D01D4DA8421FD0D3F8085312
:10112000ED061BD0D3F8085305F01F05052D15D08B
:10113000D3F8085305F01F05092D0FD0606D40F45A
:1011400080106065D868800105D5606D20F400507E
:1011500040F48050606584F8502010E0C3689B0123
:1011600005D5636D23F4005343F48053636584F81D
:101170005020826842F00402826000E002210846AA
:1011800070BD0000002002400021024000600258B3
:101190002DE9F047044640790027154601280E4600
:1011A00009D04FF0010884F80580022020713068D2
:1011B000042803D03BE00220BDE8F0874FF003098C
:1011C0001DBBFFF749F8DFF8D0A0074604E0FFF7A2
:1011D00043F8C01B012810D82068406B10EA0A0FA2
:1011E000F5D10120FFF747F82168B069086416E0DF
:1011F000FFF732F8C01B012807D9206940F008002A
:10120000206184F804900320D6E72068406B002812
:10121000EEDB0120FFF72FF82168B0694864F06920
:101220002168A8408864306A2168A840C864306991
:10123000012808D12068826B1F21A9408A43716967
:10124000A940114381632068C26B0721B368A9409C
:101250008A4331681943F3681943A9401143C163B4
:10126000206801684FF48042AA40914301602068E1
:10127000016840F6FE72AA4091437268AA400A4390
:10128000026020680168C022AA409143016084F88E
:101290000480002060718FE700800020006809B1A1
:1012A000006B7047C06A704770B5040003D02079A6
:1012B000002510B105E0012070BD2046657100F0E9
:1012C00007F802202071256101202071002070BDE7
:1012D000104800B587B0016841F000510160006816
:1012E00000F0005005900B480838016841F00101FA
:1012F00001600068694600F0010005901020009030
:1013000003200190002002900348FEF7AFFF07B0D2
:1013100000BD0000E84402580000025818B50468F7
:1013200000940068104421B1143000900360002044
:1013300018BD0830F9E730B54279012A12D00123EF
:101340004371022202710268146803FA01F52C430A
:101350001460002901680A6806D0C2F34442012AD9
:101360000AD00DE0022030BDC2F34402012A07D1A9
:101370004A6842F0010202E04A6842F002024A6012
:10138000037100214171084630BD000010B528B13D
:1013900090F83510022903D080214165012010BD4D
:1013A0001D4A4FF4956301688C189C4207D80422AB
:1013B00080F83520086820F00100086029E00C68FA
:1013C00024F00E040C6001680A440A6822F001024D
:1013D0000A60016E0A6822F480720A6090F85C303C
:1013E000012202FA03F10D4B1960D0E919134B6089
:1013F000C16E31B10B6823F480730B60D0E91C130C
:101400004B60002180F8341080F83520016D01B167
:101410008847002010BD0000F0FFFDBF04540258B3
:101420002DE9F041044690F8A00015460F4601282A
:101430001DD0012684F8A060022084F8A10005EBED
:10144000850000EBC500342204EB80003830FEF745
:1014500049FE2A463946204604F0BAFA2068466218
:1014600084F8A160002084F8A000BDE8F08102208B
:10147000FBE7000070B5040004D094F8A10000253B
:1014800010B106E0012070BD204684F8A05000F0A5
:101490006BF8022084F8A1002068816921F0704176
:1014A0008161D4E901100143D4E9030210430143EF
:1014B00020688269114381612068826829490A4055
:1014C0008260A08A020420688368A66933431343BC
:1014D00083602068C2680A40C260A08B0204206852
:1014E000C368266A33431343C360206802690A4015
:1014F0000261A08C020420680369A66A3343134387
:101500000361206842690A404261A08D010420689D
:101510004269236B1A430A43426194F83500020280
:1015200094F8360001042068C36A03F07F43C36265
:101530002068C36A114394F8346033430B43C36299
:101540002068416B41F0060141632068816941F0E8
:1015500001018161C4F8A450012084F8A100002099
:1015600070BD000000F800F02B4810B586B001688F
:1015700041F008010160006800F00800059026486D
:101580001038016841F010010160006800F010009F
:1015900005902148001F016841F4807101600168D5
:1015A00001F480710591016841F4007101600168E6
:1015B00001F400710591016841F4806101600068E7
:1015C0000324694600F480600590202000900120EB
:1015D0000190CDE902041148FEF748FE4FF4E040C7
:1015E00000900220019000206946CDE902040E20FF
:1015F00004900B48FEF73AFE48F67C6000900948DC
:101600006946FEF733FEFF20009007486946FEF763
:101610002DFE06B010BD0000E4440258000402583C
:1016200000200258002402580028025870B50446D1
:1016300090F8A0000E46012820D0012584F8A05083
:10164000022084F8A10003EB830000EBC30004EB4D
:1016500080018E63086E3044C1E90F02486E104469
:10166000486438311A46204604F0B2F920684562D1
:1016700084F8A150002084F8A00070BD022070BD45
:1016800070B5044690F8A0000E46012820D0012530
:1016900084F8A050022084F8A10003EB830000EB43
:1016A000C30004EB8001886B3044C863086C1044AD
:1016B0004864C1E9186238311A46204604F088F9B6
:1016C0002068456284F8A150002084F8A00070BD15
:1016D000022070BD10B5FEF7D3FD084909684FF42C
:1016E000807292FAA2F201F47061B2FA82F2D140F1
:1016F000034A515CC8400349086010BD18440258B1
:101700009E1900080000002410B5FEF7BEFD074931
:101710000968102292FAA2F201F07001B2FA82F284
:10172000D140034A515CC84010BD0000204402581B
:101730009E190008364930B50A68096812F003029C
:10174000344BC1F305311B68334C03F0100324689C
:10175000DFED320AB7EE001AC4F3CC0414FB03F336
:1017600000EE103A2E4BB8EE400A07D02D4C012A5D
:1017700001D0022A4AD0B4FBF1F10BE0244C283C02
:1017800022689506284A03D52468C4F3C104E240C0
:10179000B2FBF1F101EE901A1968B8EE612AC1F3BB
:1017A000080101EE901A1968F8EE611A40EE201A4D
:1017B00031EE810A22EE000AC1F34621491C00EEF7
:1017C000901AF8EE600A80EE201AFCEEC10AC0ED15
:1017D000000A1968C1F30641491C00EE901AF8EEA0
:1017E000600A80EE201AFCEEC10AC0ED010A1968F9
:1017F000C1F30661491C00EE901AF8EE600A80EE13
:10180000201ABCEEC10A80ED020A30BD074ABFE7CC
:10181000284402582C4402583C4402580000003925
:101820003844025800093D000090D00340787D0103
:10183000364930B50A68096812F00302344BC1F327
:1018400005511B68334C03F480732468DFED320AC2
:10185000B7EE001AC4F3CC0414FB03F300EE103A05
:101860002E4BB8EE400A07D02D4C012A01D0022A97
:101870004AD0B4FBF1F10BE0244C283C22689506D9
:10188000284A03D52468C4F3C104E240B2FBF1F155
:1018900001EE901A1968B8EE612AC1F3080101EE51
:1018A000901A1968F8EE611A40EE201A31EE810A9A
:1018B00022EE000AC1F34621491C00EE901AF8EE10
:1018C000600A80EE201AFCEEC10AC0ED000A196819
:1018D000C1F30641491C00EE901AF8EE600A80EE52
:1018E000201AFCEEC10AC0ED010A1968C1F30661B5
:1018F000491C00EE901AF8EE600A80EE201ABCEE49
:10190000C10A80ED020A30BD074ABFE728440258E9
:101910002C44025844440258000000394044025804
:1019200000093D000090D00340787D012DE9F84F7B
:101930000446006800252E46010104F12400FE4FF4
:10194000DFF8F88300901DD5606E50B1B0F5801FB0
:101950000CD0B0F5001F0ED0B0F5401F1DD00125F2
:101960000FE0386840F40030386016E00221201D96
:1019700004F00AF903E00098022104F07DF9050063
:101980000BD02E462088C00523D5606D05281ED2B9
:10199000DFE800F00C11161B1B00D8F80010626E77
:1019A00021F440111143C8F80010EBE7386840F407
:1019B0000030386009E00021201D04F0E5F803E064
:1019C0000098002104F058F905466DB100E00125AA
:1019D0002E432088800528D5A06D80281ED00CDCE1
:1019E00090B140280ED114E0D8F80010626D21F0BB
:1019F00007011143C8F80010EBE7C02813D0B0F579
:101A0000807F10D001250FE0386840F40030386046
:101A100009E00021201D04F0B7F803E00098002140
:101A200004F02AF9054685B12E432088DFF810938B
:101A300040052CD5D4F8A400B0F5800F20D00DDCE3
:101A4000A0B1B0F5001F0FD115E0D8F80010A26DBD
:101A500021F4E0711143C8F80010E6E7B0F5C00FBB
:101A600013D0B0F5000F10D001250FE0386840F416
:101A70000030386009E00021201D04F085F803E003
:101A80000098002104F0F8F8054675B12E4320882F
:101A900000052DD5D4F8A800B0F1007F21D00EDCD0
:101AA000A8B1B0F1807F10D116E0D9F80010D4F8B9
:101AB000A42021F460011143C9F80010E7E7B0F158
:101AC000407F13D0B0F1806F10D001250FE038684F
:101AD00040F40030386009E00021201D04F054F883
:101AE00003E00098002104F0C7F805466DB12E43CD
:101AF000206880011FD5A06CD8B110280FD02028F5
:101B000012D0302815D0012514E0D9F80010D4F8EF
:101B1000A82021F0E0611143C9F80010E8E7386817
:101B200040F40030386004E00221201D04F02CF85D
:101B300005466DB12E432088C0042BD5E06DB0F56D
:101B4000005F20D00DDCA0B1B0F5805F0FD115E0B3
:101B50007A48001F0168A26C21F030011143016036
:101B6000E9E7B0F5405F13D0B0F5804F10D0012504
:101B70000FE0386840F40030386009E00021201D93
:101B800004F002F803E00098002104F075F805461F
:101B900085B12E432088800429D5206EB0F5403FC2
:101BA00023D010DC08B3B0F5803F14D0B0F5003F6F
:101BB0000FD115E0D8F80010E26D21F4E041114397
:101BC000C8F80010E6E7B0F5802F0ED0B0F5A02FD2
:101BD0000BD001250AE00121201D03F0D5FF03E011
:101BE0000098012104F048F805468DB12E43208865
:101BF00040042AD5D4F8AC00B0F1405F23D010DC0B
:101C000008B3B0F1805F14D0B0F1005F0FD115E0E0
:101C1000D8F80010226E21F4E0211143C8F800101A
:101C2000E5E7B0F1804F0ED0B0F1A04F0BD0012509
:101C30000AE00121201D03F0A7FF03E00098012125
:101C400004F01AF805466DB12E43208800041FD514
:101C5000E06ED8B1B0F1805F0ED0B0F1005F10D06F
:101C6000012514E0D9F80010D4F8AC2021F0E041AF
:101C70001143C9F80010E8E7386840F400303860D4
:101C800004E00121201D03F07FFF05466DB12E43C6
:101C90002068C0011ED5606CD0B101280ED002288A
:101CA00011D0032814D0012513E0D8F80010E26EFB
:101CB00021F040511143C8F80010E9E7386840F4BA
:101CC0000030386004E00221201D03F05DFF05466E
:101CD00075B12E432068DFF86CB040025AD51A481F
:101CE000016841F480710160FEF7B6FA82460EE0A9
:101CF0001248001F0168626C21F00301114301606A
:101D0000E8E7FEF7A9FAA0EB0A0064283AD80E48E3
:101D10000068C005F5D5B5BB094818300068B4F8AF
:101D2000B01000F4407001F44071884219D00448AA
:101D3000183001680AE000002C4402585044025850
:101D4000584402581044025800480258026821F4CE
:101D5000407142F480320260026822F480320260F4
:101D60000160D4F8B000B0F5807F22D1FEF774FA9C
:101D7000824609E0FEF770FAA0EB0A0141F28830D2
:101D8000814201D9032504E0FE4800688007F1D5AF
:101D90007DB12E432078DFF8F0A3C0073CD0A06FC0
:101DA000182837D025DC78B3082828D0102824D16B
:101DB0002BE0D4F8B000C0F3012103290ED0DBF8EA
:101DC000001021F47C51CBF80010EE480168B4F803
:101DD000B020C2F30B0211430160DBE7DBF8002007
:101DE000EA4B22F47C5203EA10100243CBF80020A5
:101DF000EBE720280ED028280CD001250BE001218C
:101E0000201D03F0C1FE04E004E00098012103F06E
:101E100033FF05465DB12E43207880071ED5606FE5
:101E2000062819D2DFE800F0160C11161616DAF89B
:101E30000010A26F21F038011143CAF80010EBE73F
:101E40000121201D03F0A0FE03E00098012103F012
:101E500013FF054675B100E001252E4320784007A9
:101E60001FD5D4F89000062819D2DFE800F0160C30
:101E700011161616DAF80010626F21F007011143EF
:101E8000CAF80010EAE70121201D03F07DFE03E0FF
:101E90000098012103F0F0FE05469DB100E0012508
:101EA0002E43207880062BD5D4F88C00B0F1405F0B
:101EB00024D011DC10B3B0F1805F15D0B0F1005F19
:101EC00010D116E0D9F80010D4F8902021F00701C5
:101ED0001143C9F80010E4E7B0F1804F0ED0B0F123
:101EE000A04F0BD001250AE00021201D03F04CFE7D
:101EF00003E00098022103F0BFFE05468DB12E439A
:101F0000207840062BD5D4F89800B0F5406F24D047
:101F100011DC10B3B0F5806F15D0B0F5006F10D1A3
:101F200016E0DAF80010D4F88C2021F0E0411143DB
:101F3000CAF80010E4E7B0F5805F0ED0B0F5A05FFE
:101F40000BD001250AE00021201D03F01DFE03E057
:101F50000098022103F090FE05468DB12E432078B3
:101F600000062BD5D4F89C00B0F5C04F24D011DC6E
:101F700010B3B0F5005F15D0B0F5804F10D116E06A
:101F8000D9F80010D4F8982021F4E0511143C9F891
:101F90000010E4E7B0F5004F0ED0B0F5204F0BD0A5
:101FA00001250AE00021201D03F0EEFD03E000986A
:101FB000022103F061FE054665B32E432078000739
:101FC0000BD5D4F88000B0F5805F2DD0DAF8002072
:101FD00022F440520243CAF800202078C0060BD5F4
:101FE000D4F89400B0F5807F24D0D9F8002022F4F2
:101FF00040720243C9F80020206800032CD5D4F8B1
:10200000A000E8B1B0F5803F1FD0B0F5003F21D06F
:10201000012520E0D9F80010D4F89C2021F460417B
:102020001143C9F80010C9E70098022103F024FE0B
:102030000643D2E70098022103F01EFE0643DBE7C9
:102040000021201D03F0A0FD03E00098022103F011
:1020500013FE054685B12E432068400322D5D4F8EF
:102060008400B0F5801F11D0B0F5001F13D0B0F57B
:10207000401F15D0012514E0D9F80010D4F8A02095
:1020800021F440311143C9F80010E5E7386840F405
:102090000030386004E00098012103F0EDFD0546B2
:1020A00055B12E432068C0031CD5E06C70B1B0F56B
:1020B000803F10D0012514E0DAF80010D4F8842015
:1020C00021F440111143CAF80010EBE7386840F4DE
:1020D0000030386004E00221201D03F055FD054664
:1020E000C5B12E432068800004D50098022103F07A
:1020F000C3FD0643206880031BD5E06FB8B1B0F57F
:10210000807F10D0B0F5007F11D0B0F5407F0ED0A9
:1021100001250DE01C4808380168E26C21F480318B
:1021200011430160DEE7386840F40030386045B3A1
:102130002E432068C00207D5D8F80000226F20F097
:1021400000401043C8F800002068C00008D5DBF844
:102150000010D4F8B42021F480411143CBF80010D2
:102160002068800207D5D8F80010A26E21F0807197
:102170001143C8F800102068400014D5DBF80010A7
:1021800006E01EE07044025854440258CFFFFF009E
:1021900021F40041CBF80010DBF80010D4F8B8208F
:1021A0001143CBF800102068002806DA0A480168BD
:1021B000226D21F04051114301605EB10120BDE864
:1021C000F88FDAF80010E26F21F440711143CAF879
:1021D0000010AEE70020F2E74C44025870B504004E
:1021E0000D4603D094F82C0010B107E0012070BD1B
:1021F000002084F82D00204600F018F8022084F812
:102200002C002068211DFEF78FF9D4E90002294631
:10221000FEF7CAF90448016841F00041016001205D
:1022200084F82C00002070BD00400052444800B5E6
:1022300087B0016841F002010160006800F002000F
:1022400005903F482038016841F4805101600068E2
:1022500000F4805005903A481438016841F00401B8
:102260000160016801F004010591016841F0080175
:102270000160016801F008010591016841F0100159
:102280000160016801F010010591016841F0200131
:102290000160016801F020010591016841F04001F1
:1022A0000160016801F040010591016841F0800181
:1022B0000160016801F080010591016841F48071BD
:1022C00001600068694600F4807005900D20009060
:1022D0000220019001200290032003900C20049022
:1022E0001848FDF7C3FF4CF203700090164869468A
:1022F000FDF7BCFF4FF68370009014486946FDF768
:10230000B5FF4FF63F00009011486946FDF7AEFF5C
:1023100048F2371000900F486946FDF7A7FF4FF4C9
:102320007F4000900C486946FDF7A0FF40F2FF6037
:1023300000900A486946FDF799FF07B000BD00000C
:10234000F444025800080258000C025800100258C9
:102350000014025800180258001C025800200258AD
:1023600010B5044690F82C00022809D0022084F809
:102370002C002068FEF700F9012084F82C000020D2
:1023800010BD70B5044690F82C000D4602280CD004
:10239000022084F82C002068FEF7F4F82868022850
:1023A00004D0012084F82C00002070BD0520F9E73E
:1023B00070B5040015460E4603D094F8450010B1E0
:1023C00007E0012070BD002084F84400204600F0A2
:1023D00021F8206804F10801FEF73CF8A2683146B4
:1023E0002068FEF773F8E36A2946D4E90102FEF794
:1023F00011F8A168206850F8212042F0010240F84D
:1024000021200348016841F000410160002070BDB7
:10241000004000521A4800B587B0016841F480516D
:102420000160006800F48050059015480C30016888
:1024300041F008010160016801F00801059101689F
:1024400041F0100101600068694600F0100005903D
:102450004EF2B37000900220019001200290032000
:1024600003900C2004900748FDF700FF4FF68070A2
:10247000009005486946FDF7F9FE07B000BD000071
:10248000D4440258000C025800100258704770479C
:1024900090F8791090F87A000843704770B5026898
:1024A0000446D0691368916810F00F0F64D0594D3D
:1024B00003F490760D40354376D0C50707D0DD058F
:1024C00005D501251562E26F42F00102E26782073D
:1024D00008D5CA0706D0256802222A62E26F42F0B8
:1024E0000402E267420708D5CA0706D0256804221D
:1024F0002A62E26F42F00202E26702070ED503F0A1
:10250000200201F080552A4352EAC17206D02568A4
:1025100008222A62E26F42F00802E267E26F002AB4
:102520003AD0800608D503F0200001F0805108431E
:1025300002D0204603F035FDE06F000703D4206889
:10254000806840062AD5204603F01DFD206881687A
:1025500049061ED5816821F040018160606FC0B1DD
:102560002D490165606FFEF711FF002814D0606FE0
:10257000016DBDE870400847850615D503F02005BC
:1025800001F0805635430FD02046BDE8704003F07F
:1025900008BD2046FFF77BFF70BD05E02046FFF732
:1025A00076FF0020E067F7E7C6024FF020050CD564
:1025B0004E020AD5E803106284F8795084F87A5004
:1025C0002046BDE87040FFF761BF06060AD503F05C
:1025D000800601F400010E4304D02046BDE870409F
:1025E00003F06EBF41060BD5590609D51168204688
:1025F00021F04001116084F8795000F097F8CBE7A2
:102600000002C9D55800C7D5106820F0804010607E
:10261000C2E7000001000010735F009010B50400D5
:1026200003D094F8790010B107E0012010BD00201C
:1026300084F878002046FDF72DFE242084F87900E8
:102640002068016821F001010160204603F0E4FCEC
:102650000128EBD0606B10B1204603F0F8FB206836
:10266000416821F4904141602068816821F02A018D
:1026700081602068016841F0010101602046BDE8E9
:10268000104003F048BC90F87A30202B4CD1B9B1FF
:10269000B2B190F87830012B46D0012380F8783021
:1026A0004166A0F86820A0F86A20FF228168B1F591
:1026B000805F07D07F2351B1B1F1805F0CD010E073
:1026C00001207047016921B940F2FF1107E001695B
:1026D00009BBA0F86C2004E00169E1B13F21A0F83A
:1026E0006C100021C167222280F87A2080F87810CF
:1026F00001688A6842F001028A6001680A689200F3
:102700000CD50A6842F480720A600068816841F062
:102710008051816006E0A0F86C30E2E7086840F480
:102720009070086000207047022070477047FEE7F5
:102730001B4870B586B0016841F001010160016875
:1027400001F001010591016841F004010160016897
:1027500001F004010591016841F080010160006809
:1027600003240025694600F0800005900220012620
:10277000CDE902040B48CDE90065FDF777FD700354
:1027800003948DE8610008486946FDF76FFD0C2051
:10279000009006486946FDF769FD06B070BD00006F
:1027A000E04402580000025800080258001C025879
:1027B0002DE9F0470126304CDFF8C080DFF8C090EB
:1027C0007703304D01281DD02078A0B1082128467C
:1027D000FDF765FDC0B104212846FDF760FD98B105
:1027E00039464046FDF75BFD70B101214846FDF7D3
:1027F00056FD012808D008212846FDF750FD012884
:1028000026D037E02670E1E70A20FDF72AFD0020F8
:10281000207008212846FDF742FD80B1042128469A
:10282000FDF73DFD70B139464046FDF738FD58B122
:1028300001214846FDF733FD012807D01AE00120A9
:10284000BDE8F0870220FBE70320F9E70420F7E763
:1028500004212846FDF723FD01280BD139464046C7
:10286000FDF71DFD012805D101214846FDF717FDA3
:1028700000B926700020E3E7200000240008025879
:1028800000000258001C02580E490F4A70B5064657
:1028900008881268002422B13046BDE8704002F07A
:1028A000CBBD4D8800214543084602F017FC02F0DD
:1028B0008BFDB1B2054801E00180641CAC42FBD342
:1028C00070BD0000C8010024B402002400000860AC
:1028D0002DE9F05F394C3A4DA071296839B102F009
:1028E000CFFDE88A2080288B6080BDE8F09F3349C7
:1028F0002C232A254FF0F0092B2649F2413A4FF4B8
:10290000305E45F2105B89884FF448774FF4A07829
:1029100045F2103C4FF4F07258B1A4F800805145D4
:10292000A4F8029001D0614529D123816581A68157
:1029300039E0A4F800905145A4F8028001D0614527
:1029400008D1238161456581A68131D1A4F8008039
:1029500062802DE0594508D1A4F808E04FF42850D2
:1029600060814FF42C50A08106E0A1F5C850633877
:102970001ED123816681A5812280678018E0594598
:1029800008D1A4F808E04FF4285060814FF42C508F
:10299000A08106E0A1F5C850633804D12381658188
:1029A000A68127806280614502D12280A4F802803E
:1029B0000020BDE8F05F02F0B5BA0000C8010024B5
:1029C000B40200242DE9F04104463A480D4600685F
:1029D00020B12046BDE8F04102F066BD364E270A20
:1029E0004FEA15283146B0884989A0F51343413B89
:1029F0000CD0A0F5A643103B08D0A0F5AA43103B8D
:102A000011D0A0F5C853633B27D04BE0084602F035
:102A1000CFFC384602F0C0FCE0B202F0BDFCB08949
:102A200002F0C6FC38E0084602F0C2FC384602F06C
:102A3000B3FC7089401C80B202F0BAFCE0B202F034
:102A4000ABFCB08902F0B4FC404602F0A5FCB089B2
:102A5000401C80B202F0ACFC21E0B07918B930889B
:102A6000001B401E84B2084602F0A2FC270A38462A
:102A700002F092FCE0B202F08FFC384602F08CFCCF
:102A8000E0B202F089FCB08902F092FC404602F00C
:102A900083FCE8B202F080FC404602F07DFCE8B224
:102AA00002F07AFC054930890880881C0280BDE864
:102AB000F0810000B4020024C8010024FEFF07607A
:102AC0002DE9F04F95B002F025FFFE4D4FF6FF7A4D
:102AD00049F2413945F21036A5F14C0845F210543F
:102AE00041F66317A88018B102F052FD02F08DB9CB
:102AF000F548016841F00201016000680EA900F08C
:102B00000200139020200E9001200F9010900320BF
:102B10001190EE48FDF7AAFB02F0A4F9EC4910224F
:102B2000C8F800104046EB49C8F804100021C8F866
:102B30000810C8F80C10C0E904121202C8F81810E6
:102B4000C8F81C10C0E908129200C0E90A129201EC
:102B5000C8F830101120C8E90D12CDE90701552041
:102B6000099015200290CDE90001D6486A460D91E2
:102B70004C38069107A9FFF71BFC3220FDF771FBCB
:102B8000D32002F015FC02F099F9A88002F096F922
:102B9000A88002F093F90AEA00205246A88002F0C9
:102BA0008DF9A9880843A880484546D0D42002F072
:102BB000FFFB02F083F9A88002F080F9A88002F000
:102BC0007DF902EA0020A88002F078F9A98808437C
:102BD000A880B04231D04FF45A4002F0E9FB02F035
:102BE0006DF9A8804FF45B4002F0E2FB02F066F959
:102BF00002EA0020A8804FF45C4002F0D9FB02F00A
:102C00005DF9A9880843A880B0F5004F7DD0A042A7
:102C100013D0A12002F0CCFB02F050F9A88002F002
:102C20004DF902EA0020A88002F048F9A98808437B
:102C3000A880A0F5AE41613968D080B2484566D120
:102C4000CF2002F0B5FB002002F0A6FBC12002F06D
:102C5000A3FB302002F0A0FBED2002F0A9FB6420D2
:102C600002F09AFB032002F097FB122002F094FB83
:102C7000812002F091FBE82002F09AFB852002F00F
:102C80008BFB102002F088FB7A2002F085FBCB2022
:102C900002F08EFB392002F07FFB2C2002F07CFB3F
:102CA000002002F079FB342002F076FB022002F0D3
:102CB00073FBF72002F07CFB202002F06DFBEA2082
:102CC00002F076FB002002F067FB002002F064FBBC
:102CD000C02002F06DFB1B2002F05EFBC12002F061
:102CE00067FB012002F058FBC52002F061FB302099
:102CF00002F052FB302002F04FFBC72002F058FBDD
:102D0000B72002F049FB362002E0B4E0B0E0B4E0C6
:102D100002F04EFB482002F03FFB3A2002F048FB55
:102D2000552002F039FBB12002F042FB002002F0F6
:102D300033FB1A2002F030FBB62002F039FB0A20E8
:102D400002F02AFBA22002F027FBF22002F030FB67
:102D5000002002F021FB262002F02AFB012002F0D5
:102D60001BFBE02002F024FB0F2002F015FB2A20C1
:102D700002F012FB282002F00FFB082002F00CFBEF
:102D80000E2002F009FB082002F006FB542002F09E
:102D900003FBA92002F000FB432002F0FDFA0A2009
:102DA00002F0FAFA0F2002F0F7FA002002F0F4FA2B
:102DB000002002F0F1FA002002F0EEFA002002F00A
:102DC000EBFAE12002F0F4FA002002F0E5FA152017
:102DD00002F0E2FA172002F0DFFA072002F0DCFA34
:102DE000112002F0D9FA062002F0D6FA2B2002F0C8
:102DF000D3FA562002F0D0FA3C2002F0CDFA05209A
:102E000002F0CAFA102002F0C7FA0F2002F0C4FA4A
:102E10003F2002F0C1FA3F2002F0BEFA0F2002F07C
:102E2000BBFA2B2002F0C4FA002002F0B5FA002011
:102E300002F0B2FA012002F0AFFA3F2002F0ACFA41
:102E40002A2002F0B5FA002002F0A6FA002002F0D3
:102E5000A3FA002002F0A0FAEF2002F09DFA112060
:102E600002F0A6FA7820FDF7FCF9292001F010BF46
:102E7000AF8001F012BFAC80FDE3B0427ED1ED2007
:102E800002F096FA012002F087FAFE2002F084FA9E
:102E9000EE2002F08DFADE2002F07EFA212002F010
:102EA0007BFAF12002F084FA012002F075FADF20AB
:102EB00002F07EFA102002F06FFAC42002F078FAD5
:102EC0008F2009E0C8010024E044025800040258A1
:102ED000004000520441005202F05EFAC62002F0A7
:102EE00067FA002002F058FAE22002F055FAE220D8
:102EF00002F052FAE22002F04FFABF2002F058FA34
:102F0000AA2002F049FAB02002F052FA0D2002F095
:102F100043FA002002F040FA0D2002F03DFA0020B2
:102F200002F03AFA112002F037FA002002F034FAE7
:102F3000192002F031FA002002F02EFA212002F0CE
:102F40002BFA002002F028FA2D2002F025FA0020AA
:102F500002F022FA3D2002F01FFA002002F01CFAD3
:102F60005D2002F019FA002002F016FA5D2002F04E
:102F700013FA002002F010FAB12000E0FEE302F0A4
:102F800017FA802002F008FA002002F005FA8B20E0
:102F900002F002FA002002F0FFF9962002F0FCF99C
:102FA000002002F0F9F9B22002F002FA002002F04B
:102FB000F3F9002002F0F0F9022002F0EDF9002010
:102FC00002F0EAF9032002F0E7F9002002F0E4F948
:102FD000B32002F0EDF9002002F0DEF9002002F04B
:102FE000DBF9002002F0D8F9002002F0D5F900202A
:102FF00002F0D2F9002002F0CFF9002002F0CCF963
:10300000002002F0C9F9002002F0C6F9002002F009
:10301000C3F9002002F0C0F9002002F0BDF9002041
:1030200002F0BAF9002002F0B7F9002002F0B4F97A
:10303000002002F0B1F9002002F0AEF9002002F009
:10304000ABF9002002F0A8F9002002F0A5F9002059
:1030500002F0A2F9002002F09FF9002002F09CF992
:10306000002002F099F9B42002F0A2F98B2002F0BE
:1030700093F9002002F090F9962002F08DF90020DB
:1030800002F08AF9A12002F087F9002002F084F909
:10309000B52002F08DF9022002F07EF9002002F046
:1030A0007BF9032002F078F9002002F075F9042082
:1030B00002F072F9002002F06FF9B62002F078F900
:1030C000002002F069F9002002F066F9B72002F052
:1030D0006FF9002002F060F9002002F05DF93F2056
:1030E00002F05AF9002002F057F95E2002F054F97C
:1030F000002002F051F9642002F04EF9002002F0A5
:103100004BF98C2002F048F9002002F045F9AC2080
:1031100002F042F9002002F03FF9DC2002F03CF915
:10312000002002F039F9702002F036F9002002F098
:1031300033F9902002F030F9002002F02DF9EB2055
:1031400002F02AF9002002F027F9DC2002F024F92D
:10315000002002F021F9B82002F02AF9002002F044
:103160001BF9002002F018F9002002F015F90020E8
:1031700002F012F9002002F00FF9002002F00CF921
:10318000002002F009F9002002F006F9BA2002F04E
:103190000FF9242002F000F9002002F0FDF80020D1
:1031A00002F0FAF8002002F0F7F8C12002F000F96E
:1031B000202002F0F1F8002002F0EEF8542002F096
:1031C000EBF8002002F0E8F8FF2002F0E5F800201C
:1031D00002F0E2F8C22002F0EBF80A2002F0DCF87C
:1031E000002002F0D9F8042002F0D6F8002002F006
:1031F000D3F8C32002F0DCF83C2002F0CDF8002028
:1032000002F0CAF83A2002F0C7F8002002F0C4F831
:10321000392002F0C1F8002002F0BEF8372002F099
:10322000BBF8002002F0B8F83C2002F0B5F800200E
:1032300002F0B2F8362002F0AFF8002002F0ACF84D
:10324000322002F0A9F8002002F0A6F82F2002F0A8
:10325000A3F8002002F0A0F82C2002F09DF8002036
:1032600002F09AF8292002F097F8002002F094F872
:10327000262002F091F8002002F08EF8242002F0BF
:103280008BF8002002F088F8242002F085F8002056
:1032900002F082F8232002F07FF8002002F07CF890
:1032A0003C2002F079F8002002F076F8362002F097
:1032B00073F8002002F070F8322002F06DF8002060
:1032C00002F06AF82F2002F067F8002002F064F89C
:1032D0002C2002F061F8002002F05EF8292002F0B4
:1032E0005BF8002002F058F8262002F055F8002084
:1032F00002F052F8242002F04FF8002002F04CF8BF
:10330000242002F049F8002002F046F8232002F0C1
:1033100043F8002002F040F8C42002F049F862208F
:1033200002F03AF8002002F037F8052002F034F8F5
:10333000002002F031F8842002F02EF8002002F084
:103340002BF8F02002F028F8002002F025F81820D1
:1033500002F022F8002002F01FF8A42002F01CF86E
:10336000002002F019F8182002F016F8002002F0F0
:1033700013F8502002F010F8002002F00DF80C2095
:1033800002F00AF8002002F007F8172002F004F813
:10339000002002F001F8952001F0FEFF002001F06E
:1033A000FBFFF32001F0F8FF002001F0F5FFE6201D
:1033B00001F0F2FF002001F0EFFFC52001F0F8FF5F
:1033C000322001F0E9FF002001F0E6FF442001F087
:1033D000E3FF002001F0E0FF652001F0DDFF0020A9
:1033E00001F0DAFF762001F0D7FF002001F0D4FFD2
:1033F000882001F0D1FF002001F0CEFFC62001F0AF
:10340000D7FF202001F0C8FF002001F0C5FF1720E2
:1034100001F0C2FF002001F0BFFF012001F0BCFF5E
:10342000002001F0B9FFC72001F0C2FF002001F029
:10343000B3FF002001F0B0FF002001F0ADFF00203D
:1034400001F0AAFFC82001F0B3FF002001F0A4FFA3
:10345000002001F0A1FF002001F09EFF002001F0FC
:103460009BFFC92001F0A4FF002001F095FF002080
:1034700001F092FF002001F08FFF002001F08CFF8F
:10348000002001F089FF002001F086FF002001F0FC
:1034900083FF002001F080FF002001F07DFF00206D
:1034A00001F07AFF002001F077FF002001F074FFA7
:1034B000002001F071FF002001F06EFF002001F0FC
:1034C0006BFF002001F068FFE02001F071FF162083
:1034D00001F062FF002001F05FFF1C2001F05CFFA3
:1034E000002001F059FF212001F056FF002001F0DB
:1034F00053FF362001F050FF002001F04DFF462021
:1035000001F04AFF002001F047FF522001F044FF84
:10351000002001F041FF642001F03EFF002001F097
:103520003BFF7A2001F038FF002001F035FF8B20AF
:1035300001F032FF002001F02FFF992001F02CFF55
:10354000002001F029FFA82001F026FF002001F053
:1035500023FFB92001F020FF002001F01DFFC4204F
:1035600001F01AFF002001F017FFCA2001F014FF3C
:10357000002001F011FFD22001F00EFF002001F029
:103580000BFFD92001F008FF002001F005FFE0202B
:1035900001F002FF002001F0FFFEF32001F0FCFE2D
:1035A000002001F0F9FEE12001F002FF162001F0F9
:1035B000F3FE002001F0F0FE1C2001F0EDFE0020E3
:1035C00001F0EAFE222001F0E7FE002001F0E4FE17
:1035D000362001F0E1FE002001F0DEFE452001F082
:1035E000DBFE002001F0D8FE522001F0D5FE0020C5
:1035F00001F0D2FE642001F0CFFE002001F0CCFEED
:103600007A2001F0C9FE002001F0C6FE8B2001F0F7
:10361000C3FE002001F0C0FE992001F0BDFE002095
:1036200001F0BAFEA82001F0B7FE002001F0B4FEC0
:10363000B92001F0B1FE002001F0AEFEC42001F07F
:10364000ABFE002001F0A8FECA2001F0A5FE00207C
:1036500001F0A2FED22001F09FFE002001F09CFEAE
:10366000D82001F099FE002001F096FEE02001F044
:1036700093FE002000E08BE301F08EFEF32001F0CA
:103680008BFE002001F088FEE22001F091FE052073
:1036900001F082FE002001F07FFE0B2001F07CFE95
:1036A000002001F079FE1B2001F076FE002001F0E1
:1036B00073FE342001F070FE002001F06DFE442006
:1036C00001F06AFE002001F067FE4F2001F064FE69
:1036D000002001F061FE612001F05EFE002001F09B
:1036E0005BFE792001F058FE002001F055FE882095
:1036F00001F052FE002001F04FFE972001F04CFE39
:10370000002001F049FEA62001F046FE002001F055
:1037100043FEB72001F040FE002001F03DFEC22034
:1037200001F03AFE002001F037FEC72001F034FE20
:10373000002001F031FED12001F02EFE002001F02A
:103740002BFED62001F028FE002001F025FEDD2012
:1037500001F022FE002001F01FFEF32001F01CFE0C
:10376000002001F019FEE32001F022FE052001F007
:1037700013FE002001F010FE0A2000E006E301F035
:103780000BFE002001F008FE1C2001F005FE0020C9
:1037900001F002FE332001F0FFFD002001F0FCFDEE
:1037A000442001F0F9FD002001F0F6FD502001F069
:1037B000F3FD002001F0F0FD622001F0EDFD00209E
:1037C00001F0EAFD782001F0E7FD002001F0E4FDC2
:1037D000882001F0E1FD002001F0DEFD972001F0DE
:1037E000DBFD002001F0D8FDA62001F0D5FD002072
:1037F00001F0D2FDB72001F0CFFD002001F0CCFD9B
:10380000C22001F0C9FD002001F0C6FDC72001F073
:10381000C3FD002001F0C0FDD12001F0BDFD00205E
:1038200001F0BAFDD52001F0B7FD002001F0B4FD94
:10383000DD2001F0B1FD002001F0AEFDF32001F02C
:10384000ABFD002001F0A8FDE42001F0B1FD012056
:1038500001F0A2FD002001F09FFD012001F09CFD80
:10386000002001F099FD022001F096FD002001F0FA
:1038700093FD2A2001F090FD002001F08DFD3C20F9
:1038800001F08AFD002001F087FD4B2001F084FD4E
:10389000002001F081FD5D2001F07EFD002001F09F
:1038A0007BFD742001F078FD002001F075FD84207F
:1038B00001F072FD002001F06FFD932001F06CFD1E
:1038C000002001F069FDA22001F066FD002001F05A
:1038D00063FDB32001F060FD002001F05DFDBE201E
:1038E00001F05AFD002001F057FDC42001F054FD05
:1038F000002001F051FDCD2001F04EFD002001F02F
:103900004BFDD32001F048FD002001F045FDDD20F6
:1039100001F042FD002001F03FFDF32001F03CFDED
:10392000002001F039FDE52001F042FD002001F00A
:1039300033FD002001F030FD002001F02DFD0020BE
:1039400001F02AFD022001F027FD002001F024FDF6
:10395000292001F021FD002001F01EFD3C2001F096
:103960001BFD002001F018FD4B2001F015FD00208B
:1039700001F012FD5D2001F00FFD002001F00CFDB3
:10398000742001F009FD002001F006FD842001F003
:1039900003FD002001F000FD932001F0FDFC00205C
:1039A00001F0FAFCA22001F0F7FC002001F0F4FC89
:1039B000B32001F0F1FC002001F0EEFCBE2001F08C
:1039C000EBFC002001F0E8FCC42001F0E5FC002045
:1039D00001F0E2FCCD2001F0DFFC002001F0DCFC76
:1039E000D32001F0D9FC002001F0D6FCDC2001F04E
:1039F000D3FC002001F0D0FCF32001F0CDFC00202E
:103A000001F0CAFCE62001F0D3FC112001F0C4FC57
:103A1000002001F0C1FC342001F0BEFC002001F0C8
:103A2000BBFC562001F0B8FC002001F0B5FC76206C
:103A300001F0B2FC002001F0AFFC772001F0ACFCFB
:103A4000002001F0A9FC662001F0A6FC002001F096
:103A5000A3FC882001F0A0FC002001F09DFC99202F
:103A600001F09AFC002001F097FCBB2001F094FCCF
:103A7000002001F091FC992001F08EFC002001F063
:103A80008BFC662001F088FC002001F085FC5520AD
:103A900001F082FC002001F07FFC552001F07CFC4D
:103AA000002001F079FC452001F076FC002001F0B7
:103AB00073FC432001F070FC002001F06DFC4420F9
:103AC00001F06AFC002001F067FCE72001F070FCC7
:103AD000322001F061FC002001F05EFC552001F075
:103AE0005BFC002001F058FC762001F055FC002022
:103AF00001F052FC662001F04FFC002001F04CFC6C
:103B0000672001F049FC002001F046FC672001F02D
:103B100043FC002001F040FC872001F03DFC002028
:103B200001F03AFC992001F037FC002001F034FC50
:103B3000BB2001F031FC002001F02EFC992001F0A7
:103B40002BFC002001F028FC772001F025FC002050
:103B500001F022FC442001F01FFC002001F01CFCBD
:103B6000562001F019FC002001F016FC232001F082
:103B700013FC002001F010FC332001F00DFC0020AC
:103B800001F00AFC452001F007FC002001F004FCD4
:103B9000E82001F00DFC002001F0FEFB002001F008
:103BA000FBFB992001F0F8FB002001F0F5FB8720DA
:103BB00001F0F2FB002001F0EFFB882001F0ECFBAC
:103BC000002001F0E9FB772001F0E6FB002001F086
:103BD000E3FB662001F0E0FB002001F0DDFB882024
:103BE00001F0DAFB002001F0D7FBAA2001F0D4FBA2
:103BF000002001F0D1FBBB2001F0CEFB002001F042
:103C0000CBFB992001F0C8FB002001F0C5FB66202A
:103C100001F0C2FB002001F0BFFB552001F0BCFB0E
:103C2000002001F0B9FB552001F0B6FB002001F0A7
:103C3000B3FB442001F0B0FB002001F0ADFB4420B9
:103C400001F0AAFB002001F0A7FB552001F0A4FB26
:103C5000002001F0A1FBE92001F0AAFBAA2001F05D
:103C60009BFB002001F098FB002001F095FB002059
:103C700001F092FB002001F09BFBAA2001F08CFBDD
:103C8000CF2001F095FB002001F086FB002001F021
:103C900083FB002001F080FB002001F07DFB002071
:103CA00001F07AFB002001F077FB002001F074FBAB
:103CB000002001F071FB002001F06EFB002001F0FC
:103CC0006BFB002001F068FB002001F065FB002089
:103CD00001F062FB002001F05FFB002001F05CFBC3
:103CE000002001F059FB002001F056FBF02001F00C
:103CF0005FFB002001F050FB502001F04DFB002045
:103D000001F04AFB002001F047FB002001F044FBDA
:103D1000F32001F04DFB002001F03EFBF92001F003
:103D200047FB062001F038FB102001F035FB29206D
:103D300001F032FB002001F02FFB3A2001F038FBAC
:103D4000552001F029FB112001F032FB6420FCF723
:103D500088FA292001F02CFB352001F029FB0020F6
:103D600001F01AFB512001F023FBFF2001F014FBAE
:103D7000532001F01DFB2C2001F00EFB552001F01B
:103D800017FB822001F008FB2C20FDE3A0427DD12F
:103D90004FF470435521184601F020FB4FF2010B00
:103DA000AA21584601F01AFB52214FF2020001F0FD
:103DB00015FB08214FF2030001F010FB01214FF227
:103DC000040001F00BFB0D214FF4304001F006FB25
:103DD0000D214BF2010001F001FB0D214BF202001D
:103DE00001F0FCFA34214FF4364001F0F7FA3421A7
:103DF0004BF2016001F0F2FA34214BF2026001F063
:103E0000EDFA0D214FF4314001F0E8FA0D214BF2AB
:103E1000011001F0E3FA0D214BF2021001F0DEFA7D
:103E200034214FF4374001F0D9FA34214BF20170BC
:103E300001F0D4FA34214BF2027001F0CFFA0021E4
:103E40004FF4324001F0CAFA00214BF2012001F098
:103E5000C5FA00214BF2022001F0C0FA24214FF4F0
:103E6000384001F0BBFA24214BF6010001F0B6FA0C
:103E700024214BF6020001F0B1FA01214FF43F403A
:103E800001F0ACFA0F214FF4334000E0FEE301F003
:103E9000A5FA0F214BF2013001F0A0FA0F214BF2ED
:103EA000023001F09BFA34214FF4394001F096FAC8
:103EB00034214BF6011001F091FA34214BF6021037
:103EC00001F08CFA08214FF4354001F087FA0821FF
:103ED0004BF2015001F082FA08214BF2025001F03E
:103EE0007DFA03214FF4424001F078FA24214FF487
:103EF0003A4001F073FA24214BF6012001F06EFAEA
:103F000024214BF6022001F069FA00214FF43C40D5
:103F100001F064FA78214BF6014001F05FFA0021CC
:103F20004BF6024001F05AFA00214FF43D4001F0F7
:103F300055FA78214BF6015001F050FA00214BF66A
:103F4000025001F04BFA00214FF43E4001F046FAD6
:103F500064214BF6016001F041FA00214FF4514019
:103F600001F03CFA33214DF2011001F037FA002143
:103F70004DF2021001F032FA34214DF2031001F03B
:103F80002DFA00214DF2041001F028FA3A214DF2E9
:103F9000051001F023FA00214DF2061001F01EFA7F
:103FA0004A214DF2071001F019FA00214DF20810D4
:103FB00001F014FA5C214DF2091001F00FFA002112
:103FC0004DF20A1001F00AFA81214DF20B1001F0B6
:103FD00005FA00214DF20C1001F000FAA6214DF275
:103FE0000D1001F0FBF900214DF20E1001F0F6F971
:103FF000E5214DF20F1001F0F1F901214DF2101001
:1040000001F0ECF913214DF2111001F0E7F9012153
:104010004DF2121001F0E2F954214DF2131001F0AB
:10402000DDF901214DF2141001F0D8F982214DF291
:10403000151001F0D3F901214DF2161001F0CEF95F
:10404000CA214DF2171001F0C9F902214DF21810E2
:1040500001F0C4F900214DF2191001F0BFF902215D
:104060004DF21A1001F0BAF901214DF21B1001F0C6
:10407000B5F902214DF21C1001F0B0F934214DF2D6
:104080001D1001F0ABF902214DF21E1001F0A6F94E
:1040900067214DF21F1001F0A1F902214DF220100D
:1040A00001F09CF984214DF2211001F097F90221D1
:1040B0004DF2221001F092F9A4214DF2231001F0EB
:1040C0008DF902214DF2241001F088F9B7214DF24B
:1040D000251001F083F902214DF2261001F07EF93E
:1040E000CF214DF2271001F079F902214DF228106D
:1040F00001F074F9DE214DF2291001F06FF902216F
:104100004DF22A1001F06AF9F2214DF22B1001F064
:1041100065F902214DF22C1001F060F9FE214DF2FB
:104120002D1001F05BF903214DF22E1001F056F92C
:1041300010214DF22F1001F051F903214DF23010F2
:1041400001F04CF933214DF2311001F047F9032110
:104150004DF2321001F042F96D214DF2331001F0B1
:104160003DF900214FF4524001F038F933214DF26E
:10417000012001F033F900214DF2022001F02EF967
:1041800034214DF2032001F029F900214DF20420E1
:1041900001F024F93A214DF2052001F01FF9002128
:1041A0004DF2062001F01AF94A214DF2072001F0E4
:1041B00015F900214DF2082001F010F95C214DF2B3
:1041C000092001F00BF900214DF20A2001F006F957
:1041D00081214DF20B2001F001F900214DF20C205C
:1041E00001F0FCF8A6214DF20D2001F0F7F80021B6
:1041F0004DF20E2001F0F2F8E5214DF20F2001F012
:10420000EDF801214DF2102001F0E8F813214DF2F4
:10421000112001F0E3F801214DF2122001F0DEF847
:1042200054214DF2132001F0D9F801214DF2142050
:1042300001F0D4F882214DF2152001F0CFF80121D0
:104240004DF2162001F0CAF8CA214DF2172001F0F4
:10425000C5F802214DF2182001F0C0F800214DF2FE
:10426000192001F0BBF802214DF21A2001F0B6F836
:1042700001214DF21B2001F0B1F802214DF21C206A
:1042800001F0ACF834214DF21D2001F0A7F8022115
:104290004DF21E2001F0A2F867214DF21F2001F01F
:1042A0009DF802214DF2202001F098F884214DF272
:1042B000212001F093F802214DF2222001F08EF826
:1042C000A4214DF2232001F089F802214DF224208F
:1042D00001F084F8B7214DF2252001F07FF802218A
:1042E0004DF2262001F07AF8CF214DF2272001F07F
:1042F00075F802214DF2282001F070F8DE214DF210
:10430000292001F06BF802214DF22A2001F066F815
:10431000F2214DF22B2001F061F802214DF22C2008
:1043200001F05CF8FE214DF22D2001F057F8032139
:104330004DF22E2001F052F810214DF22F2001F005
:104340004DF803214DF2302001F048F833214DF2B1
:10435000312001F043F803214DF2322001F03EF804
:104360006D214DF2332001F039F800214FF4534014
:1043700001F034F833214DF2013001F02FF8002123
:104380004DF2023001F02AF834214DF2033001F0F1
:1043900025F800214DF2043001F020F83A214DF2C9
:1043A000053001F01BF800214DF2063001F016F83F
:1043B0004A214DF2073001F011F800214DF208308A
:1043C00001F00CF85C214DF2093001F007F80021F2
:1043D0004DF20A3001F002F881214DF20B3000F06D
:1043E000FDFF00214DF20C3000F0F8FFA6214DF248
:1043F0000D3000F0F3FF00214DF20E3000F0EEFF23
:10440000E5214DF20F3000F0E9FF01214DF21030AF
:1044100000F0E4FF13214DF2113000F0DFFF012125
:104420004DF2123000F0DAFF54214DF2133000F05B
:10443000D5FF01214DF2143000F0D0FF82214DF262
:10444000153000F0CBFF01214DF2163000F0C6FF11
:10445000CA214DF2173000F0C1FF02214DF2183091
:1044600000F0BCFF00214DF2193000F0B7FF02212F
:104470004DF21A3000F0B2FF01214DF21B3000F076
:10448000ADFF02214DF21C3000F0A8FF34214DF2A7
:104490001D3000F0A3FF02214DF21E3000F09EFF00
:1044A00067214DF21F3000F099FF02214DF22030BC
:1044B00000F094FF84214DF2213000F08FFF0221A3
:1044C0004DF2223000F08AFFA4214DF2233000F09B
:1044D00085FF02214DF2243000F080FFB7214DF21C
:1044E000253000F07BFF02214DF2263000F076FFF0
:1044F000CF214DF2273000F071FF02214DF228301C
:1045000000F06CFFDE214DF2293000F067FF022140
:104510004DF22A3000F062FFF2214DF22B3000F014
:104520005DFF02214DF22C3000F058FFFE214DF2CC
:104530002D3000F053FF03214DF22E3000F04EFFDE
:1045400010214DF22F3000F049FF03214DF23030A1
:1045500000F044FF33214DF2313000F03FFF0321E2
:104560004DF2323000F03AFF6D214DF2333000F061
:1045700035FF00214FF4544000F030FF33214DF25D
:10458000014000F02BFF00E082E300214DF20240E9
:1045900000F024FF34214DF2034000F01FFF002102
:1045A0004DF2044000F01AFF3A214DF2054000F0B0
:1045B00015FF00214DF2064000F010FF4A214DF298
:1045C000074000F00BFF00214DF2084000F006FF0D
:1045D0005C214DF2094000F001FF00214DF20A403C
:1045E00000F0FCFE81214DF20B4000F0F7FE0021AF
:1045F0004DF20C4000F0F2FEA6214DF20D4000F00D
:10460000EDFE00214DF20E4000F0E8FEE5214DF2F6
:104610000F4000F0E3FE01214DF2104000F0DEFEFD
:1046200013214DF2114000F0D9FE01214DF212404C
:1046300000F0D4FE54214DF2134000F0CFFE0121D2
:104640004DF2144000F0CAFE82214DF2154000F0F8
:10465000C5FE01214DF2164000F0C0FECA214DF208
:10466000174000F0BBFE02214DF2184000F0B6FEEC
:1046700000214DF2194000F0B1FE02214DF21A4026
:1046800000F0ACFE01214DF21B4000E003E300F01E
:10469000A5FE02214DF21C4000F0A0FE34214DF297
:1046A0001D4000F09BFE02214DF21E4000F096FEE0
:1046B00067214DF21F4000F091FE02214DF2204093
:1046C00000F08CFE84214DF2214000F087FE022193
:1046D0004DF2224000F082FEA4214DF2234000F072
:1046E0007DFE02214DF2244000F078FEB7214DF20C
:1046F000254000F073FE02214DF2264000F06EFED0
:10470000CF214DF2274000F069FE02214DF22840F2
:1047100000F064FEDE214DF2294000F05FFE022130
:104720004DF22A4000F05AFEF2214DF22B4000F0EB
:1047300055FE02214DF22C4000F050FEFE214DF2BC
:104740002D4000F04BFE03214DF22E4000F046FEBE
:1047500010214DF22F4000F041FE03214DF2304078
:1047600000F03CFE33214DF2314000F037FE0321D2
:104770004DF2324000F032FE6D214DF2334000F038
:104780002DFE00214FF4554000F028FE33214DF25C
:10479000015000F023FE00214DF2025000F01EFEF9
:1047A00034214DF2035000F019FE00214DF2045067
:1047B00000F014FE3A214DF2055000F00FFE0021EA
:1047C0004DF2065000F00AFE4A214DF2075000F06B
:1047D00005FE00214DF2085000F000FE5C214DF274
:1047E000095000F0FBFD00214DF20A5000F0F6FDEB
:1047F00081214DF20B5000F0F1FD00214DF20C50E3
:1048000000F0ECFDA6214DF20D5000F0E7FD002177
:104810004DF20E5000F0E2FDE5214DF20F5000F098
:10482000DDFD01214DF2105000F0D8FD13214DF2B5
:10483000115000F0D3FD01214DF2125000F0CEFDD9
:1048400054214DF2135000F0C9FD01214DF21450D6
:1048500000F0C4FD82214DF2155000F0BFFD012192
:104860004DF2165000F0BAFDCA214DF2175000F07B
:10487000B5FD02214DF2185000F0B0FD00214DF2BF
:10488000195000F0ABFD02214DF21A5000F0A6FDC8
:1048900001214DF21B5000F0A1FD02214DF21C50F0
:1048A00000F09CFD34214DF21D5000F097FD0221D7
:1048B0004DF21E5000F092FD67214DF21F5000F0A6
:1048C0008DFD02214DF2205000F088FD84214DF233
:1048D000215000F083FD02214DF2225000F07EFDB8
:1048E000A4214DF2235000F079FD02214DF2245015
:1048F00000F074FDB7214DF2255000F06FFD02214C
:104900004DF2265000F06AFDCF214DF2275000F005
:1049100065FD02214DF2285000F060FDDE214DF2D0
:10492000295000F05BFD02214DF22A5000F056FDA7
:10493000F2214DF22B5000F051FD02214DF22C508E
:1049400000F04CFDFE214DF22D5000F047FD0321FB
:104950004DF22E5000F042FD10214DF22F5000F08C
:104960003DFD03214DF2305000F038FD33214DF272
:10497000315000F033FD03214DF2325000F02EFD96
:104980006D214DF2335000F029FD00214FF45640C7
:1049900000F024FD33214DF2016000F01FFD0021E5
:1049A0004DF2026000F01AFD34214DF2036000F078
:1049B00015FD00214DF2046000F010FD3A214DF28A
:1049C000056000F00BFD00214DF2066000F006FDD1
:1049D0004A214DF2076000F001FD00214DF2086010
:1049E00000F0FCFC5C214DF2096000F0F7FC0021B6
:1049F0004DF20A6000F0F2FC81214DF20B6000F0F4
:104A0000EDFC00214DF20C6000F0E8FCA6214DF217
:104A10000D6000F0E3FC00214DF20E6000F0DEFCC2
:104A2000E5214DF20F6000F0D9FC01214DF210603C
:104A300000F0D4FC13214DF2116000F0CFFC0121F5
:104A40004DF2126000F0CAFC54214DF2136000F0E8
:104A5000C5FC01214DF2146000F0C0FC82214DF232
:104A6000156000F0BBFC01214DF2166000F0B6FCB1
:104A7000CA214DF2176000F0B1FC02214DF218601E
:104A800000F0ACFC00214DF2196000F0A7FC0221FF
:104A90004DF21A6000F0A2FC01214DF21B6000F003
:104AA0009DFC02214DF21C6000F098FC34214DF277
:104AB0001D6000F093FC02214DF21E6000F08EFCA0
:104AC00067214DF21F6000F089FC02214DF2206049
:104AD00000F084FC84214DF2216000F07FFC022173
:104AE0004DF2226000F07AFCA4214DF2236000F028
:104AF00075FC02214DF2246000F070FCB7214DF2EC
:104B0000256000F06BFC02214DF2266000F066FC8F
:104B1000CF214DF2276000F061FC02214DF22860A8
:104B200000F05CFCDE214DF2296000F057FC022110
:104B30004DF22A6000F052FCF2214DF22B6000F0A1
:104B40004DFC02214DF22C6000F048FCFE214DF29C
:104B50002D6000F043FC03214DF22E6000F03EFC7E
:104B600010214DF22F6000F039FC03214DF230602E
:104B700000F034FC33214DF2316000F02FFC0321B2
:104B80004DF2326000F02AFC6D214DF2336000F0EE
:104B900025FC5521184600F021FCAA21584600F0BA
:104BA0001DFC52214FF2020000F018FC08214FF2C8
:104BB000030000F013FC00214FF2040000F00EFC93
:104BC000CC214FF4314000F009FC00214BF20110E0
:104BD00000F004FC05214FF4364000F0FFFB70218B
:104BE0004FF4374000F0FAFB70214BF2017000F0F7
:104BF000F5FB01214FF4384000F0F0FB03214BF6A8
:104C0000010000F0EBFB03214BF6020000F0E6FB95
:104C100003214BF6030000F0E1FB02214FF43C407E
:104C200000F0DCFB00214BF6014000F0D7FB002137
:104C30004BF6024000F0D2FBD0214FF4494000F087
:104C4000CDFB02214CF6011000F0C8FB50214CF6C0
:104C5000021000F0C3FB50214CF6031000F0BEFB25
:104C600050214CF6041000F0B9FB00214FF45450D1
:104C700000F0B4FB55214FF4685000F0AFFB4FF447
:104C8000885000F095FB7820FBF70EFB4FF4245082
:104C900000F08EFBB9E0B842FCD1E22000F088FBC6
:104CA0001D2000F079FB022000F076FB042000F0CC
:104CB00073FB6420FBF7F8FAE02000F079FB012099
:104CC00000F06AFB0A20FBF7CCFAE02000F070FB52
:104CD000032000F061FB0C20FBF7C3FA012000F079
:104CE00067FB0A20FBF7BDFAE62000F061FB2F20EE
:104CF00000F052FBFF2000F04FFBFF2000F04CFBC8
:104D0000B02000F055FB202000F046FB002000F012
:104D100043FB032000F040FB40F21F3000F03CFB5F
:104D2000012000F039FB40F2DF1000F035FB0020DD
:104D300000F032FBB42000F03BFB042000F02CFB21
:104D400040F21F4000F028FB002000F025FB2E2041
:104D500000F022FB002000F01FFB002000F01CFBF5
:104D6000002000F019FB002000F016FBB62000F038
:104D70001FFB022000F010FB4FF4037000F00CFB4F
:104D8000002000F009FB172000F006FB152000F0C2
:104D900003FB002000F000FB002000F0FDFAF020F3
:104DA00000F006FB032000F0F7FA292000F000FBDA
:104DB000D02000F0FDFA002000F0EEFABE2000F056
:104DC000F7FA052000F0E8FAFE2000F0E5FA0120ED
:104DD00000F0E2FA002000F0DFFA002000F0DCFA38
:104DE000002000F0D9FAB82000F0E2FA032000F029
:104DF000D3FA012000F0D0FABA2000F0D9FA01204D
:104E000000F0CAFA642000F063F8A888484505D08D
:104E1000B04203D0A04201D0B84209D10520009091
:104E200002906946D8F82C30D8E90102FBF7F2FA73
:104E3000A98808A0FBF7EAF80020FDF749FD08481B
:104E400001222021FBF735FA5046FDF71DFD15B074
:104E5000BDE8F08F4C43442049443A25780D0A00C0
:104E6000000402581FB5FBF729FA032201218DF82F
:104E70000010500701901B208DF8080000208DF8CD
:104E80000C008DF809008DF80D008DF80A008DF8E2
:104E90000E0068468DF801208DF80B208DF80F105C
:104EA000FBF711FA0420FBF713FA1FBD034601209C
:104EB00000E05843491EC9B2FBD27047034808B509
:104EC0000088ADF80000BDF8000008BD00000860D3
:104ED0000246BE2000B500F06BFA052000F05CFA37
:104EE00000EE102A9FED0D1BB8EE400B20EE010BDB
:104EF000BCEEC00B10EE100A80B200F04DFA01209B
:104F000000F04AFAFF2000F047FA002000F044FACF
:104F10005DF804EB002000F03FBA000066666666AC
:104F200066660440F0B56C4D002341F663142946D3
:104F3000AA798988012A01D01AB11BE0A14202D1C5
:104F400018E0A14216D1082814D2DFE800F00406C8
:104F5000080A0C0E101206200CE007200AE00420BC
:104F600008E0052006E0012004E0002002E0032024
:104F700000E0022045F21032A1F5134745F2105629
:104F8000413F05D0914203D0B14201D0A14277D137
:104F9000082812D2DFE800F0110406080A0C0E10EF
:104FA00080230AE0402308E0C02306E0202304E039
:104FB000602302E0A02300E0E023B14202D14FF4DD
:104FC000585000E03620914205D0B14203D0A142B2
:104FD00001D043F00803194600F000FAAA88A24263
:104FE0000AD069889806288802D5884202D303E04F
:104FF000884201D929806880B242688941D100F095
:10500000D7F9002000F0C8F96889401C80B200F090
:10501000CFF9002000F0C0F96889801C80B200F050
:10502000C7F92888401EC0F30F2000F0B5F9688941
:10503000C01C80B200F0BCF92878401EC0B200F05D
:10504000ABF9A88900F0B4F9002000F0A5F9A8890F
:10505000401C80B200F0ACF9002000F09DF9A88956
:10506000801C80B200F0A4F96888401EC0F30F20B5
:1050700000F092F9A889C01C80B200F099F922E0F2
:1050800028E000F095F9002000F086F9002000F0FB
:1050900083F92888401EC0F30F2000F07DF928789E
:1050A000401EC0B200F078F9A88900F081F9002014
:1050B00000F072F9002000F06FF96888401EC0F31C
:1050C0000F2000F069F9A878BDE8F040401EC0B29A
:1050D00000F062B9F0BD0000C8010024F0B53F4DFA
:1050E000060A0C4602462846270AA9884089A1F5E7
:1050F0001343413B28D0A1F5A643103B24D0A1F592
:10510000C853633B2FD0A1F5AA43103B64D100F0F4
:105110004FF9304600F040F96889401C80B200F039
:1051200047F9D0B200F038F9A88900F041F93846C3
:1051300000F032F9A889401C80B200F039F9E0B2E1
:10514000BDE8F04000F028B900F032F9304600F038
:1051500023F9D0B200F020F9A88900F029F93846E7
:1051600000F01AF9EBE7A97929B300F021F93046EC
:1051700000F012F9D0B200F00FF92888401EC0F3F9
:105180000F2000F009F92878401EC0B200F004F9A1
:10519000A88900F00DF9384600F0FEF8E0B200F002
:1051A000FBF86888401EC0F30F2000F0F5F8A878DF
:1051B000401EC0B2C4E72988891A491E8AB200F08D
:1051C000F7F8002000F0E8F8002000F0E5F8100AF9
:1051D00000F0E2F8D0B2D9E7F0BD0000C801002429
:1051E0002DE9F84F1F460E4682468B46580700D0E1
:1051F0000120790800EBD700203A10FB01F00025D0
:1052000002F0FF09C0B2009047E00C2F10D0102F21
:1052100012D0182F14D0202F42D1224901EBC910EF
:105220004FF00008445D200610D51F48026811E0C9
:105230001E4909EB490006E01D4901EB0910EFE7A3
:105240001C4909EBC90001EB8000E9E70A9828B97D
:105250001548426831465046FDF7B4FB6006761C9F
:10526000040E1548B6B24088B04219D9A6EB0B001F
:10527000B84209D10AF101005E461FFA80FA0E48D1
:10528000018851450CD906E008F1010000F0FF0843
:10529000B8F1080FC7D36D1CEDB200988542B4D3A6
:1052A000BDE8F88F707D009024000024B065009068
:1052B000246A009014700090C80100242DE9F84F72
:1052C00000F0FF08044610190D461FFA80FA4FF04F
:1052D000000B58191FFA80F9DDE90A7611E05445F0
:1052E00002D3E819444685B24D450FD23B462946C4
:1052F0002046CDF800B0FFF773FF04EB570084B2EF
:10530000761C3278A2F120005E28E8D9BDE8F88F3B
:105310002DE9FF4F81B080464FF000091F469346AC
:105320004C460E98DDF83CA046080AF001052BE03B
:10533000381B401EC1B20A20FFF7B8FDBBFBF0F0DE
:105340000A21B9F1000FB0FBF1F201FB120005D107
:10535000791E8C4202DA48B14FF001090E9B3030C1
:105360000095C2B206FB048080B208E05FEA0A60E2
:105370000E9B06FB0480009580B20AD5302202996C
:10538000FFF72EFF641CE4B2BC42D1D305B0BDE8E8
:10539000F08F2022F3E7000001B5BDF80000ADF862
:1053A0000000BDF800000149088008BD0000086049
:1053B00001B5BDF80000ADF80000BDF800000149DE
:1053C000088008BDFEFF0760024803490089088085
:1053D00070470000C8010024FEFF0760024A1080E9
:1053E000901C018070470000FEFF0760104810B558
:1053F00086B0016841F002010160006801210D4C96
:1054000000F0020005900320CDE90001CDE9021073
:1054100069462046FAF72AFF012220461146FAF78C
:1054200048FF012220460221FAF743FF06B010BDD3
:10543000E04402580004025808B500900548018B6A
:10544000C08A491E8BB2401E82B20021084600F07D
:1054500049F808BDB402002400B5AFB04FF00053C6
:105460000093CDE9090102200B90CDE90C026846BA
:10547000FCF75CFA002800D001202FB000BD00002E
:10548000084B10B51C465875A1888AB2218889B28C
:1054900020B1012801D1D9821A8310BDDA82198383
:1054A00010BD0000B4020024F0B50C4F94B2DFF838
:1054B00030C03D467E7D2B68EA692D7D5CF8255025
:1054C00026B103FB01004243AC52F0BD7E68301AA6
:1054D000401E03FB001050432C52F0BDB4020024C8
:1054E0002C0000242DE9F043254E0024DDF81C900B
:1054F000757D0DB1054606E077680D46B91A1A4666
:105500003B1A491E5B1E3068521B96F814C0DFF828
:105510007480871A00FB0150F6697F1E58F82CC072
:10552000BFB206FB00C51848066846F400060660D0
:1055300016484FF440360660022646630764066844
:1055400026F001060660C563591A4FF48033491CE2
:1055500003EB024211434164C0F83890016841F006
:1055600001010160420202E0641C944202D24168DF
:105570008907F9D5816841F002018160BDE8F083B7
:10558000B40200242C000024D84402580010005219
:105590002DE9FF5F00F0BEF9B84D0123082704464E
:1055A0000626A0F5864042384FF4F0723AD0A4F5B2
:1055B000E0404FF0170A84384FF4487140D0032080
:1055C0004FF08C09A4F5E04CBCF1160C4FF4806B45
:1055D0004FF4167E42D0A4F5E048B8F118084FF415
:1055E000A06C47D0A4F50048B8F1160845D0A4F542
:1055F0008058B8F1180843D04AF2010844454FF4E6
:10560000407949D140F25651C5E900198F212981CD
:1056100046212982D521A98168811821E9811C228E
:105620006882ADE04FF48870C5E900202B81282006
:105630006B81A8810520EF81582228826F829FE02C
:10564000C5E900122B812E206B81A881D220A5F8FC
:105650000EA0288216201822688291E0C5E900BEBB
:10566000142129816881A020A5F80C90E981288265
:105670000C2055E0C5E900C186E0C5E900BE83E025
:10568000C5E900C1A5F80C900A21298210222981C0
:10569000E9816982688173E0A4F52048B8F10208C5
:1056A00016D0A4F52048B8F103081FD0A4F5204C6B
:1056B000BCF1040C29D0A4F52040053833D0A4F562
:1056C000204006383ED0A4F52040073849D05BE0A2
:1056D000C5E900C120212981302129825021A981D9
:1056E0006E810E21E9811622688249E0C5E900C970
:1056F000202129815021A981302129820721698116
:105700000C21E981172268823AE0C5E900B98821B5
:10571000298118212982A021A9816E811D21E98179
:10572000122268822CE04FF45470C5E90002702008
:105730002881A881102028822F226F81A5F80EA031
:105740006E821DE0C5E9001E802028815820A881B6
:105750002820288204206881A5F80EA028226B82C8
:105760000EE04FF42070C5E90002602028812F82EE
:105770003820A881022068812921E9813E2268829F
:10578000A0210520FFF768FE3D484FF000082A6879
:105790003D4F3E4B0280696841800220E8613948F4
:1057A00038603648A838C0E90038C0F80880A4F549
:1057B0008053C0F80C80183BC0F8108002D14FF025
:1057C000805303612C89631E43616B89A3F1010C33
:1057D000C0F818C0B5F80CC06444A4F1010CC0F8BE
:1057E0001CC0B5F80EC06344A3F1010CC0F820C082
:1057F000A2F1010CA444C0F824C0A1F1010C9C4406
:10580000C0F828C0B5F810C062442244521EC262DB
:105810006A8A11441944491E016380F8368080F871
:10582000358080F834801548A838FBF723FE072020
:10583000CDE90086CDE902083968FF230222002065
:1058400000F028F8A8880022114680B2009028882D
:1058500083B2104600F04CF80020FFF711FE0C4810
:105860000122202185F81480FAF723FD04B04FF0BF
:10587000FF30BDE8F05FFFF7DFBD0000B402002499
:10588000C8010024000000C02C00002400100050BB
:10589000000402582DE9F0438DB0164614AA134DAA
:1058A00000240DF1240E92E88013009402942A68DB
:1058B00001926D68CDE904634FEA08230395CDE9B1
:1058C00006734FEA092308938EE82600024607482C
:1058D0008DF8324069468DF83140A8388DF830C0D7
:1058E000FBF79EFD0DB0BDE8F0830000B40200247C
:1058F00070B51E46044603460548049DFBF796FE18
:1059000023462A4631460248BDE87040FBF7B8BE40
:105910000C0200242B4830B587B0016841F40071B7
:105920000160016801F400710591016841F4806132
:10593000016000686946244C00F4806005904020B6
:10594000009000200190032003902046FAF78EFC7F
:105950001E4D4420694600902846FAF787FC4021F6
:105960002046FAF79CFC042104462846FAF797FCE7
:1059700044EA400428464021FAF791FC44EA8000BA
:1059800010F0FF000CD001280DD002280ED0032803
:105990000FD0042810D0052811D0002007B030BD4A
:1059A00044F24230FAE747F28400F7E747F2160084
:1059B000F4E747F21800F1E748F21600EEE741F28B
:1059C0001800EBE7E044025800240258002802586F
:1059D000F0B504688B88E568C5F30B452B441D04BE
:1059E000882303EBC213E65806F47046E6500468B9
:1059F0000F68E668C6F30B46761C3E442E43E6501D
:105A000003688C89DD68C5F30A052C4425048C24C1
:105A100004EBC2141E5906F470461E5103688F68C9
:105A2000DE68C6F30A06761C3E442E431E51046807
:105A3000942303EBC213E55825F00705E5500568EC
:105A40000C69EC5091F8313005681F0291F8323042
:105A50001C040B7E1E069C2303EBC21355F803C0E7
:105A60004FF0000C45F803C091F8305034433D43EB
:105A700025430468E5500468982303EBC213E558F6
:105A800025F0FF05E55005684C69EC500468A0233B
:105A900003EBC213E55840F20776B543E550D1E970
:105AA00007452C430568EC500468AC2303EBC21394
:105AB000E55844F803C005684C6AEC500B698BB399
:105AC000012B32D0042B32D0022B30D0032B2ED01E
:105AD000072B2CD001230568B02404EBC2142E59E7
:105AE00006F0E0262E51D1E90065AD1B0E8D5D4319
:105AF0005E43ED1D45EA064305682B510468B42357
:105B000003EBC213E5586FF30A05E5500468C96A50
:105B1000E1500068842101EBC211425842F00102B9
:105B20004250F0BDFFE70423D5E70323D3E7022368
:105B3000D1E7000012480422104910B501604FF46B
:105B40004031416000218160C0E9031201750122EA
:105B5000417582610177C0E90812816280F83820BE
:105B60001203026380F83910C162FBF797F8002234
:105B70000348BDE810401146FAF7A9BD00200240D5
:105B8000D4020024704770472DE9F047DFF8E48025
:105B900004460F464FF00009D8F80000C0438007C4
:105BA00009D0344D283D286820F080602860FAF73D
:105BB00053FB064607E00120BDE8F087FAF74CFBEF
:105BC000801B02284ED828680001F7D4D8F80010AE
:105BD000226821F47C3141EA0231C8F80010207AB1
:105BE0004FF4FE02A1884002491EA0F5007080B269
:105BF000C1F308010843A189491E02EA0141084393
:105C0000217C1202491E02EA016108431949103140
:105C100008601848001D0168626921F0C001114345
:105C200001600168A26921F02001114301606FB198
:105C30000168012F0ED041F400110160286840F086
:105C400080602860FAF708FB04460DE0016841F423
:105C50000021F2E741F48011EFE7FAF7FDFA001BAB
:105C6000022801D90320A7E728680001F5D5484696
:105C7000A2E70000284402582DE9F047DFF8E4804D
:105C800004460F464FF00009D8F80000C0438007D3
:105C900009D0344D283D286820F080502860FAF75C
:105CA000DBFA064607E00120BDE8F087FAF7D4FAF0
:105CB000801B02284ED828688000F7D4D8F800103E
:105CC000228821F07C7141EA0251C8F80010207A44
:105CD0004FF4FE02A1884002491EA0F5007080B278
:105CE000C1F308010843A189491E02EA01410843A2
:105CF000217C1202491E02EA016108431949183148
:105D000008601848001D0168626921F44061114370
:105D100001600168A26921F40071114301606FB153
:105D20000168012F0ED041F080710160286840F0B9
:105D300080502860FAF790FA04460DE0016841F4BB
:105D40008001F2E741F40001EFE7FAF785FA001B62
:105D5000022801D90320A7E728688000F5D5484626
:105D6000A2E70000284402581548012200B5134953
:105D700087B0202301600021C0E901120822C0E998
:105D80000323402343615301C0E906311302036238
:105D90005302C0E90931062102200090CDE901211A
:105DA000CDE903100590694606900548FCF716FA00
:105DB000034800F007F807B000BD00004041005262
:105DC000D8010024002301221846114610B500F026
:105DD00021F84FF4FA70FAF767FA00230122184607
:105DE000022100F017F8002308221846032100F0D2
:105DF00011F8012240F222230421002000F00AF8C9
:105E0000BDE81040024840F2A521FCF7A9BA000005
:105E1000D80100241FB5002410B1012802D002E0EF
:105E2000102400E008240748CDE902234FF6FF7252
:105E3000CDE900146946FCF7A4FA002800D001203F
:105E400004B010BDD80100247047FAF746BA90F8A4
:105E50003410C90706D001684A68836B22F4003207
:105E60001A434A6090F83410890706D501684A68D9
:105E7000C36B22F480321A434A6090F83410490709
:105E800006D501684A68036C22F480221A434A60EE
:105E900090F83410090706D501684A68436C22F46B
:105EA00000421A434A6090F83410C90606D50168CA
:105EB0008A68836C22F480521A438A6090F8341006
:105EC000890606D501688A68C36C22F400521A4319
:105ED0008A6090F83410490611D501684A68036D4C
:105EE00022F480121A434A60016DB1F5801F06D179
:105EF00001684A68436D22F4C0021A434A6090F870
:105F00003410090606D501684A68806D22F4002223
:105F100002434A607047F8B500250446C567FAF7A2
:105F20009BF90746206800686FF07E46000708D599
:105F300000223B464FF400112046009600F0FAFA8A
:105F400060B92068006840070AD500223B464FF43C
:105F500080012046009600F0EDFA08B10320F8BD5C
:105F6000202084F8790084F87A00002084F87850A2
:105F7000F8BD10B5806B0021A0F86A10A0F862107F
:105F8000FCF785FA10BD01680A6822F490720A6075
:105F900001688A6822F001028A60202180F87A1064
:105FA000704710B5B0F86C2090F87A300168222B59
:105FB00005D0088B40F008000883022010BD898CB2
:105FC0008368B3F5805F01D103696BB11140426E04
:105FD000531C43661170B0F86A10491E0904090C7D
:105FE000A0F86A1007D015E0436E11401980416E89
:105FF000891C4166EFE701680A6822F490720A6022
:1060000001688A6822F001028A60202180F87A10F3
:10601000FAF768F9002010BD2DE9F04F044600683A
:106020008025FD4B0021D4F810C087B0A6680F462C
:10603000D4F81C8046EA0C06D4F814C0A26A4CEAD4
:10604000080C46EA0C0632430668DFF8D0C306EABD
:106050000C061643066020684268E66822F4405247
:10606000324342602268A0699A4201D0266A3043D6
:10607000A66AB6F1005F04D1D4E90B6C46EA0C06BF
:1060800030439668DFF898C306EA0C06064396602C
:106090002068C26A666A22F00F023243C262E14E91
:1060A0002068E14AB04210D1126802F03802182A82
:1060B00074D005DCCAB3082A7AD0102A47D179E017
:1060C000202A7BD0282A7CD17AE0D84EB04209D150
:1060D000126802F00702062A73D2DFE802F0536961
:1060E0006B6D6F71D24EB04209D1126802F0070297
:1060F000062A66D2DFE802F0465C5E606264CD4E3E
:10610000B04209D1126802F00702062A59D2DFE82C
:1061100002F0394F51535557C74EB0420BD1126858
:1061200002F00702062A4CD200E00EE0DFE802F09F
:106130002A4042444648C14EB04209D1126802F09A
:106140003802182A38D0BBDCB4E74FF0010538E03C
:10615000BB4EB04209D1126802F00702062A30D2C3
:10616000DFE802F01026282A2C2EB64EB0420BD1C2
:10617000126802F00702062A23D2DFE802F00319B0
:106180001B1D1F2100251CE098421AD1A64A121D92
:10619000126802F00702062A13D202E00CE007E0C0
:1061A0000CE0DFE802F0030507090B0D022508E00B
:1061B000042506E0402504E0082502E0102500E063
:1061C0002025DFF864B2A04E9842DFF880A2ABF140
:1061D000540B73D1102D31D006DC022D09D0042DC3
:1061E0000AD0082D2FD111E0202D29D0402D2AD101
:1061F00007E0FBF789FA13E06846FBF79BFA019882
:106200000EE003A8FBF714FB049809E0DBF800108C
:106210005846890610D50068C0F3C1012AFA01F07A
:10622000002811D06168894601EB410181420AD8FA
:10623000B0EB093F07D808E05046F3E78448F1E7A0
:106240004FF40040EEE7012733E1102D4FF0000836
:106250004ED006DC022D0FD0042D15D0082D04D110
:106260002DE0202D4AD0402D13D00127794AA0F5EA
:106270004071914270D9E6E7FBF746FA626A002363
:10628000414636F812200DE06846FBF753FA0198B4
:1062900003E003A8FBF7CCFA04980023616A36F800
:1062A00011201946FAF723F862680902030241EA4D
:1062B00010615008181841EB080115E032E0DBF8D6
:1062C00000105846890609D500680023C0F3C101B3
:1062D0002AFA01F0616A36F8112015E0606A00239D
:1062E00036F8102050460FE00023FAF700F8BDE71B
:1062F000606A002336F81020554805E0606A0023E4
:1063000036F810204FF400400021F9F7F0FF0902A1
:10631000020241EA10614FEA590010184A4641EB67
:106320000801E1E7E3694FF4004293424DD1082DA3
:1063300023D005DC8DB1012D12D0042D06D112E041
:10634000102D35D0202D3AD0402D11D0012721F02D
:106350000F00C1F3420108435AE0F9F7CDFF16E000
:10636000F9F7CFFF13E06846FBF7E4F901980EE078
:1063700003A8FBF75DFA049809E0DBF80010584623
:10638000890608D50068C0F3C1012AFA01F0616AE4
:1063900036F8111010E0606A36F81010BAFBF1F010
:1063A0004100606801EB5001B1FBF0F081B2CEE733
:1063B000606A36F810102648B0FBF1F0F0E7606A2A
:1063C00036F81000B2FBF0F0EAE7082D4AD00ADCFC
:1063D0000DB3012D43D0042D7FF44DAF6846FBF77C
:1063E000A9F9019809E0102D52D0202D55D0402D4B
:1063F000F2D103A8FBF71CFA0498616A36F8111071
:10640000B0FBF1F1606801EB5001B1FBF0F080B23C
:106410002168C8604DE01FE0000C0058F369FFCF11
:10642000FFF4FF11001001405444025800440040A2
:1064300000480040004C0040005000400014014063
:1064400000780040007C0040986500900090D003E8
:1064500000093D00FFFC0F00F9F74EFFCDE7F9F70B
:1064600050FFCAE7DBF80020594692060AD50968B2
:10647000C1F3C1022AFA02F1626A36F81220B1FBB6
:10648000F2F20FE0616A36F81120BAFBF2F209E08D
:10649000616A36F811200949F1E7616A36F811108E
:1064A000B2FBF1F2616802EB5102B2FBF1F189B289
:1064B000C16007B03846BDE8F08F000000093D001C
:1064C00090F87910212901D002207047B0F86210AD
:1064D00021B18168B1F5805F13D014E001680A68CA
:1064E000920004D58A6822F400028A6003E00A68F8
:1064F00022F080020A600068016841F040010160FA
:106500000CE0016961B1C16D4A1CC265026809787D
:106510001185B0F86210491EA0F862100020704783
:10652000C16D02680988C1F308011185C16D891C1C
:10653000C165EEE72DE9F0411E4617468846044640
:10654000069D1CE0681C1AD025B1F9F785FE801B5A
:10655000A84214D92068016821F4D0710160206834
:10656000816821F001018160202084F8790084F89D
:106570007A00002084F878000320BDE8F0812068CC
:10658000C16938EA010004D00020B842DAD0002006
:10659000F3E70120F9E7FEE701000200040006002E
:1065A00008000A000C0010002000400080000001DC
:1065B00000000000000000000000000000000000DB
:1065C0003F400000000000000000300040003000AC
:1065D0004000000009000BC03D000BC03D00090059
:1065E00018C024407FE0224031800000180024C001
:1065F0001B000D803240018003801C4027401C801E
:106600000740004010006000000000000000000093
:106610000000000000001F802040402000004020BB
:1066200020401F8000000000090006001F800600B7
:1066300009000000040004003F8004000400000082
:1066400000100060000000000000000004000400D2
:1066500004000400040000000000004000000000EE
:1066600000000000002001C00600380040000000CB
:106670001F802040204020401F800000000010406C
:106680003FC000400000000018C0214022402440CC
:106690001840000010802040244024401B8000004F
:1066A00002000D0011003FC0014000003C8024406A
:1066B00024402440238000001F8024402440344094
:1066C000038000003000200027C0380020000000B8
:1066D0001B802440244024401B8000001C0022C05A
:1066E000224022401F8000000000000008400000FF
:1066F0000000000000000000046000000000000036
:10670000000004000A001100208040400900090038
:10671000090009000900000000004040208011002D
:106720000A00040018002000234024001800000084
:106730001F802040274029401F400000004007C024
:1067400039000F0001C0004020403FC024402440D9
:106750001B8000001F80204020402040308000002F
:1067600020403FC0204020401F80000020403FC00C
:1067700024402E4030C0000020403FC024402E0066
:10678000300000000F0010802040224033800200C3
:1067900020403FC0040004003FC020402040204073
:1067A0003FC02040204000000060202020203FC04B
:1067B0002000200020403FC024400B0030C020407B
:1067C00020403FC020400040004000C03FC03C008F
:1067D00003C03C003FC0000020403FC00C402300ED
:1067E0003FC020001F802040204020401F8000002C
:1067F00020403FC024402400180000001F8021409A
:10680000214020E01FA0000020403FC0244026007F
:1068100019C0004018C024402440224031800000AC
:10682000300020403FC020403000000020003F806A
:10683000004000403F80200020003E0001C00700D3
:1068400038002000380007C03C0007C038000000B6
:10685000204039C0060039C02040000020003840E8
:1068600007C0384020000000304021C0264038409A
:1068700020C00000000000007FE040204020000019
:10688000000070000C000380004000000000402069
:1068900040207FE0000000000000200040002000B9
:1068A0000000000000100010001000100010001088
:1068B0000000000040000000000000000000028016
:1068C0000540054003C0004020003FC00440044094
:1068D00003800000000003800440044006400000E4
:1068E00000000380044024403FC0004000000380BB
:1068F0000540054003400000000004401FC0244044
:1069000024402000000002E00550055006500420FD
:1069100020403FC00440040003C000400000044089
:1069200027C000400000000000100010041027E005
:106930000000000020403FC00140070004C00440A8
:10694000204020403FC000400040000007C004003D
:1069500007C0040003C00000044007C00440040056
:1069600003C0004000000380044004400380000096
:10697000041007F00450044003800000000003806E
:106980000440045007F00010044007C00240040017
:1069900004000000000006400540054004C000005F
:1069A000000004001F800440004000000400078035
:1069B0000040044007C000400400070004C00180FC
:1069C00006000400060001C0070001C00600000028
:1069D000044006C0010006C0044000000410071077
:1069E00004E00180060004000000044005C00640E9
:1069F000044000000000000004007BE04020000094
:106A0000000000000000FFF0000000000000402037
:106A10007BE00400000000004000800040002000F7
:106A20002000400000000000000000000000000006
:106A3000000000000000000000001FCC000C00005F
:106A40000000000000000800300060000800300076
:106A500060000000022003FC1E20022003FC1E2018
:106A60000220000000000E1811043FFF10840C7873
:106A7000000000000F0010840F3800C00778188451
:106A80000078000000780F8410C411240E9800E4F0
:106A9000008400080800680070000000000000008A
:106AA0000000000000000000000007E018182004AB
:106AB00040020000000040022004181807E0000017
:106AC000000000000240024001800FF001800240FF
:106AD000024000000080008000800FF800800080ED
:106AE000008000000001000D000E0000000000000A
:106AF0000000000000000080008000800080008016
:106B0000008000800000000C000C0000000000006D
:106B10000000000000000006001800600180060070
:106B200018002000000007F00808100410040808EE
:106B300007F000000000080408041FFC0004000423
:106B40000000000000000E0C1014102410441184EA
:106B50000E0C000000000C1810041104110412881F
:106B60000C700000000000E00320042408241FFC37
:106B70000024000000001F981084110411041088E4
:106B800010700000000007F0088811041104188834
:106B90000070000000001C00100010FC13001C001E
:106BA0001000000000000E381144108410841144BD
:106BB0000E38000000000700088C104410440888BC
:106BC00007F00000000000000000030C030C0000B0
:106BD00000000000000000000001010600000000AD
:106BE000000000000000008001400220041008089E
:106BF00010040000022002200220022002200220B5
:106C000002200000000010040808041002200140C7
:106C10000080000000000E001200100C106C1080AC
:106C20000F00000003E00C1813E4142417C4082814
:106C300007D000000004003C03C41C40074000E4EF
:106C4000001C000410041FFC1104110411040E8820
:106C50000070000003E00C18100410041004100869
:106C60001C10000010041FFC10041004100408087D
:106C700007F0000010041FFC1104110417C41004D5
:106C80000818000010041FFC1104110017C01000A8
:106C90000800000003E00C181004100410441C78D5
:106CA0000040000010041FFC10840080008010844D
:106CB0001FFC10040000100410041FFC100410043A
:106CC0000000000000030001100110011FFE100071
:106CD0001000000010041FFC110403801464181C31
:106CE0001004000010041FFC100400040004000441
:106CF000000C000010041FFC1F0000FC1F001FFC04
:106D00001004000010041FFC0C04030000E0101825
:106D10001FFC100007F008081004100410040808F5
:106D200007F0000010041FFC1084108010801080F9
:106D30000F00000007F0081810241024101C080A87
:106D400007F2000010041FFC1104110011C01130E3
:106D50000E0C000400000E1C11041084108410445A
:106D60001C3800001800100010041FFC1004100054
:106D70001800000010001FF81004000400041004A4
:106D80001FF8100010001E0011E0001C007013809E
:106D90001C0010001FC0103C00E01F0000E0103C71
:106DA0001FC000001004180C163401C001C01634B6
:106DB000180C100410001C00130400FC13041C0029
:106DC000100000000804101C1064108413041C043C
:106DD000101800000000000000007FFE400240028A
:106DE00040020000000030000C0003800060001C26
:106DF0000003000000004002400240027FFE00004D
:106E000000000000000000002000400040004000A2
:106E1000200000000001000100010001000100014C
:106E200000010001000040004000200000000000C0
:106E300000000000000000980124014401440144C6
:106E400000FC000410001FFC0088010401040088FD
:106E500000700000000000700088010401040104BB
:106E6000008800000000007000880104010411087F
:106E70001FFC0004000000F80144014401440144E7
:106E800000C800000000010401040FFC11041104FB
:106E900011001800000000D601290129012901C9AB
:106EA0000106000010041FFC008401000100010421
:106EB00000FC000400000104190419FC0004000493
:106EC000000000000000000300010101190119FE8B
:106ED0000000000010041FFC0024004001B4010C5D
:106EE000010400000000100410041FFC0004000452
:106EF00000000000010401FC0104010001FC010488
:106F0000010000FC010401FC0084010001000104F7
:106F100000FC0004000000F8010401040104010465
:106F200000F80000010101FF008501040104008850
:106F300000700000000000700088010401040105D9
:106F400001FF00010104010401FC008401040100AF
:106F500001800000000000CC012401240124012450
:106F60000198000000000100010007F8010401047D
:106F700000000000010001F8000400040004010802
:106F800001FC0004010001800170000C0010016090
:106F90000180010001F0010C003001C00030010C43
:106FA00001F0010000000104018C00740170018CEB
:106FB00001040000010101810171000E001801604F
:106FC0000180010000000184010C013401440184AE
:106FD000010C0000000000000000000001003EFC69
:106FE000400240020000000000000000FFFF00001F
:106FF000000000000000400240023EFC01000000D2
:1070000000000000000060008000800040004000A0
:107010002000200000000000000000000000000030
:107020000000000000000000000000000000000060
:107030000000000000000000000000000000000050
:10704000000000000000000F80380FFE380F80386D
:107050000000000000000000000000000000000030
:1070600000000100000600000C00003800003100A4
:10707000000600000C000038000030000000000096
:107080000000000061800067F807F980006180005F
:1070900061800061800061800067F807F98000610D
:1070A0008000000000000000000001C0E003E0F0EC
:1070B0000630080418081FFFFE040E080787F003B7
:1070C00081E000000000000001F000060C00040454
:1070D00008060C7001F9C0000E00003BE000EC183F
:1070E000070808040C180003E00000000001E0009D
:1070F00007F003F818041C0804170807E1D003C0C0
:10710000E00023B0003C0800200800001000000050
:107110000000000100003100003200001C000000EF
:10712000000000000000000000000000000000005F
:10713000000000000000000000000000000000004F
:10714000000000007F0001FFC00780F00C00181055
:1071500000042000020000000000002000021000D7
:10716000040C00180780F001FFC0007F0000000041
:10717000000000000000000000000000000000000F
:107180004200006600006600003C0000180003FF9B
:10719000C0001800003C00006600006600004200CD
:1071A00000000000080000080000080000080000BF
:1071B000080001FFC00008000008000008000008E7
:1071C0000000080000000000000100003100003253
:1071D00000001C0000000000000000000000000093
:1071E000000000000000000000000000080000088F
:1071F0000000080000080000080000080000080067
:107200000008000008000008000000000000000066
:1072100000000000380000380000380000000000C6
:10722000000000000000000000000000000000005E
:1072300000000000000600001C000070000180003B
:107240000E0000380000C0000700001C00003000E5
:1072500000000000000000007F8001FFE00380705C
:1072600006001804000804000806001803807001D6
:10727000FFE0007F8000000000000000000001002F
:107280000801000801000803FFF807FFF8000008E4
:1072900000000800000800000000000000000001DD
:1072A000C03802C0580400980401180402180404ED
:1072B00018061C1803F81801E0F800000000000090
:1072C00000000001C0E003C0F00400080408080446
:1072D000080806180803F41801E7F00001E00000B0
:1072E00000000000000000000300000D000011007D
:1072F00000610000810803010807FFF80FFFF80094
:1073000001080001080000000000000000E007FC88
:10731000D0060808061008061008061008061838D7
:10732000060FF00607C0000000000000000000008B
:107330003F8001FFE00384300208180410080410A5
:1073400008041008071810030FF00007C000000021
:1073500000000000000003C0000700000600000657
:1073600000F80607F806180006E00007000006000F
:107370000000000000000001E1E003F7F006341017
:10738000041808041808040C08040C08061618034E
:10739000F3F001C1E000000000000000F80003FC71
:1073A000300306380402080402080402080404102A
:1073B0000308F001FFC0007F000000000000000093
:1073C00000000000000000000000000070380070A5
:1073D00038007038000000000000000000000000CD
:1073E000000000000000000000000000000000009D
:1073F000301A00301C0000000000000000000000F7
:107400000000000000000000000000080000140060
:1074100000220000410000808001004002002004A2
:1074200000100800080000000000000021000021FA
:1074300000002100002100002100002100002100A7
:1074400000210000210000210000000000000000D9
:107450000000080008040010020020010040008025
:10746000800041000022000014000008000000001D
:1074700000000003C00004C0000400000800380839
:107480000F380808380810000C300007E00003C06F
:1074900000000000000000003F8000FFE00380705B
:1074A000020F1006708804C088048308047F8802D5
:1074B000C09003012000FE400000080000180001F9
:1074C000F8003E0801C20007020007E20000FE00CB
:1074D000001FC80001F80000380000080400080779
:1074E000FFF807FFF804080804080804080804085F
:1074F0000806180803F41801E7F00001E000000096
:10750000000000003F8001FFE003807002001804CB
:10751000000804000804000804001006002007808A
:10752000C000000004000807FFF807FFF804000887
:107530000400080400080400180200100380700111
:10754000FFE0007F8000000004000807FFF807FF4D
:10755000F8040808040808040808040808043E0899
:10756000040008060018010060000000040008077D
:10757000FFF807FFF80408080408000408000408DE
:1075800000043E000600000600000180000000002C
:10759000000000003F8001FFE00380700600180437
:1075A00000080402080402080203F00783F0000246
:1075B0000000020004000807FFF807FFF8040808AD
:1075C0000008000008000008000008000408080780
:1075D000FFF807FFF80400080000000000000400A6
:1075E0000804000804000807FFF807FFF804000873
:1075F0000400080400080000000000000000000073
:10760000000600000700000104000104000104005E
:107610000307FFFE07FFFC04000004000004000055
:1076200004000807FFF807FFF8040C080018000022
:107630003E0004C7800503C80600F80400380400B3
:107640001800000804000807FFF807FFF804000806
:107650000000080000080000080000080000080002
:10766000001800006000000004000807FFF8078011
:107670000807FC00007FC00003F80007C000780086
:1076800007800807FFF807FFF80400080400080750
:10769000FFF807000803C00000E000003800001EEB
:1076A000000007000001C00400F007FFF80400001C
:1076B000000000007F8001FFE003807006001804D6
:1076C000000804000806001803003001FFE0007FF6
:1076D0008000000004000807FFF807FFF804040812
:1076E000040400040400040400040400060C000365
:1076F000F80001F000000000000000007F8001FFA2
:10770000E00380700600880400880400C806003C7E
:1077100003003E01FFE6007F84000000040008072C
:10772000FFF807FFF8040808040800040C00040F21
:1077300000040BC00610F003F03801E00800000858
:1077400000000001E0F803F03006301004180804CF
:107750001808040C08040C080206180207F0078138
:10776000E0000000018000060000040000040000AA
:1077700004000807FFF807FFF804000804000004ED
:10778000000006000001800004000007FFE007FF82
:10779000F0040018000008000008000008000008BD
:1077A00000000804001007FFE004000004000006C9
:1077B000000007E00007FE00041FE00001F80000E1
:1077C000380001E0043E0007C0000600000400008D
:1077D00004000007E00007FFC0041FF80007C0070F
:1077E000F80007FF80043FF80007C004F800070016
:1077F0000004000000000004000806001807C0781C
:1078000005F1C8003E00001F800463E80780F80609
:1078100000180400080000000400000600000780B3
:107820000007E008047C08001FF80007F8001808AB
:1078300004E008070000060000040000000000014A
:1078400000080600380400F80403E8040F08047C6C
:107850000805F00807C008070018040060000000D1
:107860000000000000000000000000000000003FD9
:10787000FFFE200002200002200002200002200063
:1078800002000000000000000000080000070000E7
:1078900000C0000038000006000001C000003000F9
:1078A000000E0000010000000000000000002000A9
:1078B000022000022000022000022000023FFFFE02
:1078C00000000000000000000000000000000000B8
:1078D0000000000000080000100000300000200040
:1078E0000030000010000008000000000000000050
:1078F0000000010000010000010000010000010083
:107900000001000001000001000001000001000072
:107910000100000100000000000000000020000045
:107920002000001000001000000000000000000017
:1079300000000000000000000000000000F000193E
:10794000F8001B1800220800260800240800241054
:10795000003FF8001FF800000800001800000004B5
:10796000000007FFF80FFFF00018180010080020B3
:1079700008002008003018001FF0000FC0000000B1
:107980000000000007C0001FF000183000200800B1
:107990002008002008003C08001C100000600000C7
:1079A000000000000000000007C0001FF0003818B1
:1079B00000200800200800200804101007FFF80F1E
:1079C000FFF00000100000000000000000000007B1
:1079D000C0001FF000123000221800220800220808
:1079E000003208001E10000E200000000000000001
:1079F000200000200800200801FFF803FFF80620FF
:107A000008042008042008072000030000000000EC
:107A100000000000000E000E6E001FF30031B100E8
:107A200020B10020B1003191001F13002E1E002054
:107A30000E00300000000004000807FFF80FFFF8F8
:107A4000001008002000002000002008003FF8007F
:107A50001FF80000080000000000000000000020E7
:107A600008002008002008063FF8063FF80000083C
:107A700000000800000800000000000000000000F6
:107A8000000000000300000300200100200100208E
:107A900003063FFE063FFC0000000000000000005F
:107AA00000000004000807FFF80FFFF8000188003D
:107AB0000300002FC00038F8002038002008000024
:107AC0000800000000000000000004000804000896
:107AD00004000807FFF80FFFF80000080000080086
:107AE0000008000000000000002008003FF8003FF0
:107AF000F8001008002000003FF8003FF8001008D0
:107B0000002000003FF8003FF800000800000000DF
:107B10002008003FF8003FF8001008001000002087
:107B200000002008003FF8001FF8000008000000D7
:107B30000000000007C0000FF000183000300800FF
:107B40002008002008003008001830000FF000075F
:107B5000C0000000000000002001003FFF003FFFC8
:107B60000010110020090020080020080030380013
:107B70001FF0000FC00000000000000007C0001F41
:107B8000F00038180020080020080020090010111B
:107B9000001FFF003FFF0000010000000020080060
:107BA0002008002008003FF8003FF80008080010F7
:107BB0000800200800200000300000300000000015
:107BC000000000000000000C78001E1800330800C0
:107BD00023080021080021880021980030F0003897
:107BE00060000000000000002000002000002000D5
:107BF00000FFF003FFF80020080020080020080024
:107C00000030000000000000000000002000003FE5
:107C1000F0007FF8000018000008000008002010A5
:107C2000003FF8007FF0000010000000000000009E
:107C30002000003000003C00003F800023F00000E6
:107C400078000070002380003C000030000020001D
:107C5000002000003C00003FE00023F80000E000AE
:107C60002700003E00003FE00021F80001E0003E58
:107C70000000200000000000200800200800383824
:107C8000003E680027800003C8002CF80038380048
:107C90002018002008000000000000002000003034
:107CA00003003C01003F830023EC000070002380B0
:107CB000003C000020000020000000000000000048
:107CC00000000038080020380020F80023E8002FCA
:107CD00088003E08003808002018000070000000EE
:107CE0000000000000000000000000000000000094
:107CF00008000014001FF7FC3000062000020000FE
:107D00000000000000000000000000000000000073
:107D1000000000000000FFFFFF0000000000000066
:107D20000000000000000000000000000000200033
:107D3000023000061FF7FC001400000800000000DD
:107D4000000000000000000000000000000000181B
:107D50000000600000400000400000200000100013
:107D6000000800000400000400000C0000100000E7
:107D70000000000000000000000000000000000003
:107D800000000000000000000000000000000000F3
:107D900000000000000000000000000000000000E3
:107DA00000000000000000000000000000000000D3
:107DB00000000000000000000000000000000000C3
:107DC00000000000000000000000000000000000B3
:107DD00000000000000000000000000000000000A3
:107DE0000000000000000000000000000000000093
:107DF0000000000000000000000000000000000083
:107E0000000000000000000007F000C007FFE1E0F4
:107E100007F001E0000000C00000000000000000CA
:107E20000000000000000000000000000000000052
:107E30000000000000000000000000000000000042
:107E40000000000000000000000000000000000032
:107E50000000000000000000000000000000000022
:107E60000000000000000000000000000000000012
:107E700000000000000000000020000001C0000021
:107E8000078000001F0000001E0000001C200000F2
:107E900001C00000078000001F0000001E0000005D
:107EA0001C000000000000000000000000000000B6
:107EB00000000000000000000000000000000000C2
:107EC00000000000000000000000000000000000B2
:107ED00000000000000000000000000000000000A2
:107EE0000000000000000000000000000000000092
:107EF0000000000000180C0000180C0000180FE033
:107F0000001FFC0003F80C0000180C0000180C0007
:107F100000180C0000180C0000180FE0001FFC00F7
:107F200003F80C0000180C0000180C000000000002
:107F30000000000000000000000000000000000041
:107F40000000000000000000000000000000000031
:107F50000000000000000000000000000000000021
:107F60000000000000000000000000000000000011
:107F7000000000000000000000000780007807C03B
:107F800000FC0640010E00200307002002038020B1
:107F90000FFFFFFC0201C0200200E06001307040D2
:107FA00001F03F8000F01F00000000000000000012
:107FB00000000000000000000000000000000000C1
:107FC00000000000000000000000000000000000B1
:107FD00000000000000000000000000000000000A1
:107FE0000000000000000000000000000000000091
:107FF00000FE000001FF000003018000020080601D
:10800000030181C001FF070000FE18000000E0002E
:108010000003BF00000CFFC00071806001C10020A0
:10802000030180600000FFC000003F00000000006E
:108030000000000000000000000000000000000040
:108040000000000000000000000000000000000030
:108050000000000000000000000000000000000020
:108060000000000000000000000000000000000010
:1080700000001F0000007FC000FCC0C001FF806046
:108080000303E0200202782002061E2003FC0740C2
:1080900001F00380000103C000011C600001E0202A
:1080A00000010020000100400000018000000000ED
:1080B00000000000000000000000000000000000C0
:1080C00000000000000000000000000000000000B0
:1080D00000000000000000000000000000000000A0
:1080E0000000000000000000000000000000000090
:1080F00000000000002000001C6000001C40000088
:108100001F8000000F0000000000000000000000C1
:10811000000000000000000000000000000000005F
:10812000000000000000000000000000000000004F
:10813000000000000000000000000000000000003F
:10814000000000000000000000000000000000002F
:10815000000000000000000000000000000000001F
:10816000000000000000000000000000000000000F
:1081700000000000000000000000000000000000FF
:108180000000000000000000000000000007F800F0
:10819000003FFF00007807C001C000E0030000308E
:1081A00004000008080000041000000200000000A5
:1081B00000000000000000000000000000000000BF
:1081C00000000000000000000000000000000000AF
:1081D000000000000000000000000000000000009F
:1081E000000000000000000000000000000000008F
:1081F0000000000010000002080000040400000855
:108200000300003001C000E0007807C0003FFF001D
:108210000007F8000000000000000000000000005F
:10822000000000000000000000000000000000004E
:10823000000000000000000000000000000000003E
:10824000000000000000000000000000000000002E
:10825000000000000000000000000000000000001E
:10826000000000000000000000000000000000000E
:108270000000000000000000000C1800000E380094
:10828000000E3800000630000003600000614380EB
:1082900000FFFF8000614300000360000006300023
:1082A000000E3800000E3800000C1800000000001E
:1082B00000000000000000000000000000000000BE
:1082C00000000000000000000000000000000000AE
:1082D000000000000000000000000000000000009E
:1082E000000000000000000000000000000000008E
:1082F000000000000000000000008000000080007E
:10830000000080000000800000008000000080006D
:10831000007FFF000000800000008000000080005F
:1083200000008000000080000000800000000000CD
:10833000000000000000000000000000000000003D
:10834000000000000000000000000000000000002D
:10835000000000000000000000000000000000001D
:10836000000000000000000000000000000000000D
:108370000000000000000001000000E3000000E237
:10838000000000FC00000078000000000000000079
:1083900000000000000000000000000000000000DD
:1083A00000000000000000000000000000000000CD
:1083B00000000000000000000000000000000000BD
:1083C00000000000000000000000000000000000AD
:1083D000000000000000000000000000000000009D
:1083E000000000000000000000000000000000008D
:1083F00000000000000080000000800000008000FD
:10840000000080000000800000008000000080006C
:10841000000080000000800000008000000080005C
:1084200000008000000080000000800000000000CC
:10843000000000000000000000000000000000003C
:10844000000000000000000000000000000000002C
:10845000000000000000000000000000000000001C
:10846000000000000000000000000000000000000C
:108470000000000000000000000000C0000001E05B
:10848000000001E0000000C000000000000000004B
:1084900000000000000000000000000000000000DC
:1084A00000000000000000000000000000000000CC
:1084B00000000000000000000000000000000000BC
:1084C00000000000000000000000000000000000AC
:1084D000000000000000000000000000000000009C
:1084E000000000000000000000000000000000008C
:1084F000000000000000000C00000038000000E058
:108500000000038000000E00000038000000E000C2
:1085100000038000000E00000038000000E00000B2
:10852000038000000E0000001800000000000000A2
:10853000000000000000000000000000000000003B
:10854000000000000000000000000000000000002B
:10855000000000000000000000000000000000001B
:10856000000000000000000000000000000000000B
:108570000000000000000000000FF800007FFF0076
:1085800000F00780018000C00300006002000020AE
:10859000020000200200002003000060018000C0F3
:1085A00000E00380007FFF00000FF80000000000E3
:1085B00000000000000000000000000000000000BB
:1085C00000000000000000000000000000000000AB
:1085D000000000000000000000000000000000009B
:1085E000000000000000000000000000000000008B
:1085F00000000000000000000000000000800020DB
:1086000000800020008000200080006001FFFFE06B
:1086100003FFFFE0000000600000002000000020D9
:10862000000000200000000000000000000000002A
:10863000000000000000000000000000000000003A
:10864000000000000000000000000000000000002A
:10865000000000000000000000000000000000001A
:10866000000000000000000000000000000000000A
:108670000000000000000000007800E000980160A9
:108680000100026002000460020008600200106045
:1086900002002060020040600300806001830060EF
:1086A00001FE00E0007C07800000000000000000E8
:1086B00000000000000000000000000000000000BA
:1086C00000000000000000000000000000000000AA
:1086D000000000000000000000000000000000009A
:1086E000000000000000000000000000000000008A
:1086F000000000000000000000F0078001F007C04B
:1087000001000040020000200201002002010020C0
:1087100002010020030380200186804001FCC0C0CC
:1087200000787F8000001E000000000000000000B4
:108730000000000000000000000000000000000039
:108740000000000000000000000000000000000029
:108750000000000000000000000000000000000019
:108760000000000000000000000000000000000009
:108770000000000000000800000038000000480071
:108780000001880000060800000C081000300810E6
:108790000040081001FFFFF003FFFFF003FFFFF0B0
:1087A0000000081000000810000008100000000081
:1087B00000000000000000000000000000000000B9
:1087C00000000000000000000000000000000000A9
:1087D0000000000000000000000000000000000099
:1087E0000000000000000000000000000000000089
:1087F000000000000000000000000780001F86400D
:1088000003E10020030200200304002003040020F1
:10881000030400200304002003060040030301C0FA
:108820000301FF8003007E00000000000000000044
:108830000000000000000000000000000000000038
:108840000000000000000000000000000000000028
:108850000000000000000000000000000000000018
:108860000000000000000000000000000000000008
:1088700000000000000000000007FC00003FFF00B7
:108880000070C380008180C00101006003020020ED
:108890000202002002020020020200200203004027
:1088A00001C180C000C0FF8000007E000000000009
:1088B00000000000000000000000000000000000B8
:1088C00000000000000000000000000000000000A8
:1088D0000000000000000000000000000000000098
:1088E0000000000000000000000000000000000088
:1088F000000000000000000000F0000003C00000C5
:108900000380000003000000030007E003003FE0D5
:108910000301C0000306000003180000036000000C
:1089200003800000030000000000000000000000C1
:108930000000000000000000000000000000000037
:108940000000000000000000000000000000000027
:108950000000000000000000000000000000000017
:108960000000000000000000000000000000000007
:108970000000000000001F0000783F8000FC60C085
:10898000018EC040030780200203002002018020E6
:10899000020180200201C0200301E040018670C076
:1089A00000FC3F8000781F00000000000000000075
:1089B00000000000000000000000000000000000B7
:1089C00000000000000000000000000000000000A7
:1089D0000000000000000000000000000000000097
:1089E0000000000000000000000000000000000087
:1089F00000000000003F000000FF81C001C0C1C0B6
:108A0000010060200200202002002020020020201F
:108A100002002060020040C00100C18000C18F0040
:108A2000007FFE00001FF0000000000000000000BA
:108A30000000000000000000000000000000000036
:108A40000000000000000000000000000000000026
:108A50000000000000000000000000000000000016
:108A60000000000000000000000000000000000006
:108A700000000000000000000000000000000000F6
:108A80000000000000000000000300C0000781E0BB
:108A9000000781E0000300C00000000000000000AB
:108AA00000000000000000000000000000000000C6
:108AB00000000000000000000000000000000000B6
:108AC00000000000000000000000000000000000A6
:108AD0000000000000000000000000000000000096
:108AE0000000000000000000000000000000000086
:108AF0000000000000000000000000000000000076
:108B0000000000000000000000060066000600787B
:108B10000000000000000000000000000000000055
:108B20000000000000000000000000000000000045
:108B30000000000000000000000000000000000035
:108B40000000000000000000000000000000000025
:108B50000000000000000000000000000000000015
:108B60000000000000000000000000000000000005
:108B70000000000000000000000080000001C000B4
:108B80000003600000063000000C180000180C0004
:108B9000003006000060030000C0018001000040BA
:108BA000020000200400001000000000000000008F
:108BB00000000000000000000000000000000000B5
:108BC00000000000000000000000000000000000A5
:108BD0000000000000000000000000000000000095
:108BE0000000000000000000000000000000000085
:108BF0000000000000041000000410000004100039
:108C00000004100000041000000410000004100014
:108C10000004100000041000000410000004100004
:108C20000004100000041000000410000000000008
:108C30000000000000000000000000000000000034
:108C40000000000000000000000000000000000024
:108C50000000000000000000000000000000000014
:108C60000000000000000000000000000000000004
:108C700000000000000000000400001002000020BE
:108C80000100004000C001800060030000300600C9
:108C900000180C00000C18000006300000036000F3
:108CA0000001C00000008000000000000000000083
:108CB00000000000000000000000000000000000B4
:108CC00000000000000000000000000000000000A4
:108CD0000000000000000000000000000000000094
:108CE0000000000000000000000000000000000084
:108CF00000000000000000000078000001F8000003
:108D00000238000002000000040000C0040079E006
:108D1000040081E0040100C004030000020200001E
:108D20000306000001FC000000F800000000000045
:108D30000000000000000000000000000000000033
:108D40000000000000000000000000000000000023
:108D50000000000000000000000000000000000013
:108D60000000000000000000000000000000000003
:108D700000000000000FF800003FFE0000700780B8
:108D800000C000C00101F8400307FC20021E0420BF
:108D90000230082002203020023FFC20013F044026
:108DA00001800CC000E03180001FC2000000000004
:108DB00000000000000000000000000000000000B3
:108DC00000000000000000000000000000000000A3
:108DD0000000000000000000000000000000000093
:108DE0000000000000000000000000000000000083
:108DF0000000002000000060000003E000003E20B2
:108E00000003E020003E200003E02000038020005B
:108E100007FC2000003FE0000003FE2000003FE0D0
:108E2000000001E000000020000000200000000021
:108E30000000000000000000000000000000000032
:108E40000000000000000000000000000000000022
:108E50000000000000000000000000000000000012
:108E60000000000000000000000000000000000002
:108E700000000000020000200200002003FFFFE0CD
:108E800003FFFFE002010020020100200201002098
:108E900002010020020100200303002001868060FF
:108EA00001FCC0C000F87F8000001F00000000002F
:108EB00000000000000000000000000000000000B2
:108EC00000000000000000000000000000000000A2
:108ED0000000000000000000000000000000000092
:108EE0000000000000000000000000000000000082
:108EF000000000000007F800003FFF00007007803E
:108F000000C000C00100004003000020020000205B
:108F100002000020020000200200002001000040AA
:108F2000018000C003C00180003006000000000086
:108F30000000000000000000000000000000000031
:108F40000000000000000000000000000000000021
:108F50000000000000000000000000000000000011
:108F60000000000000000000000000000000000001
:108F700000000000020000200200002003FFFFE0CC
:108F800003FFFFE00200002002000020020000209A
:108F9000020000200300006001000040018000C0CA
:108FA00000F00780007FFE00000FF80000000000C6
:108FB00000000000000000000000000000000000B1
:108FC00000000000000000000000000000000000A1
:108FD0000000000000000000000000000000000091
:108FE0000000000000000000000000000000000081
:108FF00000000000020000200200002003FFFFE04C
:1090000003FFFFE002010020020100200201002016
:10901000020100200201002002038020020FE02054
:109020000300006003C000E00060030000000000D7
:109030000000000000000000000000000000000030
:109040000000000000000000000000000000000020
:109050000000000000000000000000000000000010
:109060000000000000000000000000000000000000
:1090700000000000020000200200002003FFFFE0CB
:1090800003FFFFE0020100200201002002010000B6
:109090000201000002010000020100000203800042
:1090A000030FE0000300000003C0000000600000A8
:1090B00000000000000000000000000000000000B0
:1090C00000000000000000000000000000000000A0
:1090D0000000000000000000000000000000000090
:1090E0000000000000000000000000000000000080
:1090F000000000000007F800003FFE00007007803D
:1091000001C001C001000040030000200200002057
:109110000200002002000020010020200100204069
:1091200003C03F8000303F8000002000000020008E
:10913000000000000000000000000000000000002F
:10914000000000000000000000000000000000001F
:10915000000000000000000000000000000000000F
:1091600000000000000000000000000000000000FF
:10917000020000200200002003FFFFE003FFFFE0E9
:10918000020080200200802000008000000080009B
:1091900000008000020080200200802003FFFFE02A
:1091A00003FFFFE00200002002000020000000009A
:1091B00000000000000000000000000000000000AF
:1091C000000000000000000000000000000000009F
:1091D000000000000000000000000000000000008F
:1091E000000000000000000000000000000000007F
:1091F000000000000000000000000000020000204D
:1092000002000020020000200200002003FFFFE017
:1092100003FFFFE002000020020000200200002007
:10922000020000200000000000000000000000001C
:10923000000000000000000000000000000000002E
:10924000000000000000000000000000000000001E
:10925000000000000000000000000000000000000E
:1092600000000000000000000000000000000000FE
:10927000000000000000000E0000000F0000000FC2
:1092800000000001020000010200000102000003D2
:109290000200000603FFFFFC03FFFFF802000000CE
:1092A00002000000020000000200000000000000B8
:1092B00000000000000000000000000000000000AE
:1092C000000000000000000000000000000000009E
:1092D000000000000000000000000000000000008E
:1092E000000000000000000000000000000000007E
:1092F00000000000020000200200002003FFFFE049
:1093000003FFFFE00200C0200201002000078000F0
:10931000000FE0000030F80002603E2003800F20C4
:10932000030003E0020000E0020000200000002033
:10933000000000000000000000000000000000002D
:10934000000000000000000000000000000000001D
:10935000000000000000000000000000000000000D
:1093600000000000000000000000000000000000FD
:1093700000000000020000200200002003FFFFE0C8
:1093800003FFFFE002000020020000200000002098
:10939000000000200000002000000020000000204D
:1093A00000000060000000E000000300000000007A
:1093B00000000000000000000000000000000000AD
:1093C000000000000000000000000000000000009D
:1093D000000000000000000000000000000000008D
:1093E000000000000000000000000000000000007D
:1093F000020000200200002003FFFFE003E0002045
:1094000003FF0020001FF0000001FF8000000FE0BC
:1094100000001E000003E000003E002003E00020EA
:1094200003FFFFE003FFFFE0020000200200002036
:10943000000000000000000000000000000000002C
:10944000000000000000000000000000000000001C
:10945000000000000000000000000000000000000C
:1094600000000000000000000000000000000000FC
:10947000020000200200002003FFFFE00380002024
:1094800003F0002000FC0000001F00000007C000E7
:109490000001F00000007C0002001F80020007E0D5
:1094A00003FFFFE0020000000200000000000000D7
:1094B00000000000000000000000000000000000AC
:1094C000000000000000000000000000000000009C
:1094D000000000000000000000000000000000008C
:1094E000000000000000000000000000000000007C
:1094F00000000000000FF800003FFE0000F00780B1
:10950000018000C001000040020000200200002095
:10951000020000200200002001000040018000C085
:1095200000F00380003FFE00000FF8000000000084
:10953000000000000000000000000000000000002B
:10954000000000000000000000000000000000001B
:10955000000000000000000000000000000000000B
:1095600000000000000000000000000000000000FB
:1095700000000000020000200200002003FFFFE0C6
:1095800003FFFFE002008020020080200200800034
:1095900002008000020080000200800003018000C1
:1095A0000183000000FE0000007C000000000000BD
:1095B00000000000000000000000000000000000AB
:1095C000000000000000000000000000000000009B
:1095D000000000000000000000000000000000008B
:1095E000000000000000000000000000000000007B
:1095F00000000000000FF800007FFF0000F0038073
:10960000018001C001000640020004200200042085
:1096100002000620020003E0010000F80180005C67
:1096200000E0038C003FFF0C000FFC18000000005E
:10963000000000000000000000000000000000002A
:10964000000000000000000000000000000000001A
:10965000000000000000000000000000000000000A
:1096600000000000000000000000000000000000FA
:1096700000000000020000200200002003FFFFE0C5
:1096800003FFFFE002010020020100200201800030
:109690000201E0000201FC0003033F80018607E0B5
:1096A00001FC00E000F800200000002000000000A5
:1096B00000000000000000000000000000000000AA
:1096C000000000000000000000000000000000009A
:1096D000000000000000000000000000000000008A
:1096E000000000000000000000000000000000007A
:1096F00000000000000000000078060000FE01E00D
:10970000018600C003030040020300200201802004
:10971000020180200201C0200200C0200100E060A0
:10972000018070C003E03F8000001F0000000000C7
:109730000000000000000000000000000000000029
:109740000000000000000000000000000000000019
:109750000000000000000000000000000000000009
:1097600000000000000000000000000000000000F9
:109770000000000000600000038000000300000003
:1097800002000000020000200200002003FFFFE0B2
:1097900003FFFFE0020000200200002002000000A2
:1097A000020000000380000000E000000000000054
:1097B00000000000000000000000000000000000A9
:1097C0000000000000000000000000000000000099
:1097D0000000000000000000000000000000000089
:1097E0000000000000000000000000000000000079
:1097F000020000000200000003FFFF0003FFFFC0A3
:109800000200004002000060000000200000002074
:109810000000002000000020020000400200008044
:1098200003FFFF0002000000020000000000000033
:109830000000000000000000000000000000000028
:109840000000000000000000000000000000000018
:109850000000000000000000000000000000000008
:1098600000000000000000000000000000000000F8
:1098700000000000020000000200000003C0000021
:1098800003FC0000023FC0000003F80000007F80DE
:10989000000007E000000780000078000203C0001D
:1098A000023C000003C000000200000002000000B3
:1098B00000000000000000000000000000000000A8
:1098C0000000000000000000000000000000000098
:1098D0000000000000000000000000000000000088
:1098E0000000000000000000000000000000000078
:1098F0000200000003C0000003FF8000023FFE00E2
:1099000002007FE000000F000200F00003EF000003
:1099100003FF8000020FFE0000003FE000001F0078
:109920000207E00003F8000003000000020000004E
:109930000000000000000000000000000000000027
:109940000000000000000000000000000000000017
:109950000000000000000000000000000000000007
:1099600000000000000000000000000000000000F7
:10997000000000000200002002000020038000E040
:1099800003F0032002FC0C20021F30000007C0007F
:109990000007F00002187C0002601F20038003E033
:1099A000020000E002000020000000200000000093
:1099B00000000000000000000000000000000000A7
:1099C0000000000000000000000000000000000097
:1099D0000000000000000000000000000000000087
:1099E0000000000000000000000000000000000077
:1099F00000000000020000000300000003C000009F
:109A000003F80000023E0020020FC0200001FFE02A
:109A100000007FE000038020021C00200270000094
:109A200003800000020000000200000000000000AF
:109A30000000000000000000000000000000000026
:109A40000000000000000000000000000000000016
:109A50000000000000000000000000000000000006
:109A600000000000000000000000000000000000F6
:109A70000000000000000020006000E0038003E020
:109A800003000FA002003E200200F8200203E020A5
:109A9000020F8020023E00200278002003E00060D8
:109AA000038000E00200030000000000000000004E
:109AB00000000000000000000000000000000000A6
:109AC0000000000000000000000000000000000096
:109AD0000000000000000000000000000000000086
:109AE0000000000000000000000000000000000076
:109AF0000000000000000000000000000000000066
:109B000000000000000000001FFFFFFC1000000428
:109B100010000004100000041000000410000004F5
:109B2000100000041000000400000000000000000D
:109B30000000000000000000000000000000000025
:109B40000000000000000000000000000000000015
:109B50000000000000000000000000000000000005
:109B600000000000000000000000000000000000F5
:109B700000000000000000000000000007000000DE
:109B800003C0000000780000001E00000003C000B9
:109B90000000F00000001E0000000780000000F040
:109BA0000000003C00000006000000000000000073
:109BB00000000000000000000000000000000000A5
:109BC0000000000000000000000000000000000095
:109BD0000000000000000000000000000000000085
:109BE0000000000000000000000000000000000075
:109BF000000000000000000010000004100000043D
:109C00001000000410000004100000041000000404
:109C1000100000041FFFFFFC000000000000000017
:109C20000000000000000000000000000000000034
:109C30000000000000000000000000000000000024
:109C40000000000000000000000000000000000014
:109C50000000000000000000000000000000000004
:109C600000000000000000000000000000000000F4
:109C700000000000000000000000000000000000E4
:109C800002000000040000000800000018000000AE
:109C90001000000018000000180000000400000080
:109CA00002000000000000000000000000000000B2
:109CB00000000000000000000000000000000000A4
:109CC0000000000000000000000000000000000094
:109CD0000000000000000000000000000000000084
:109CE0000000000000000000000000000000000074
:109CF0000000000100000001000000010000000160
:109D0000000000010000000100000001000000014F
:109D1000000000010000000100000001000000013F
:109D2000000000010000000100000001000000012F
:109D30000000000000000000000000000000000023
:109D40000000000000000000000000000000000013
:109D50000000000000000000000000000000000003
:109D600000000000000000000000000000000000F3
:109D700000000000000000000000000010000000D3
:109D80001000000010000000180000000800000093
:109D900004000000000000000000000000000000BF
:109DA00000000000000000000000000000000000B3
:109DB00000000000000000000000000000000000A3
:109DC0000000000000000000000000000000000093
:109DD0000000000000000000000000000000000083
:109DE0000000000000000000000000000000000073
:109DF000000000000000038000018FC000038C60A1
:109E00000006182000041020000410200004202068
:109E100000042040000620400003FFC00001FFE0D6
:109E20000000002000000020000000C00000000032
:109E30000000000000000000000000000000000022
:109E40000000000000000000000000000000000012
:109E50000000000000000000000000000000000002
:109E600000000000000000000000000000000000F2
:109E700000000000020000000200000003FFFFE0FD
:109E800007FFFFC0000180C0000200600002002048
:109E90000004002000040020000400200006004010
:109EA000000300C00001FF800000FE000000000071
:109EB00000000000000000000000000000000000A2
:109EC0000000000000000000000000000000000092
:109ED0000000000000000000000000000000000082
:109EE0000000000000000000000000000000000072
:109EF000000000000000000000007E000001FF8064
:109F0000000381C000020040000600200004002081
:109F10000004002000040020000600200003C040D0
:109F20000001C080000003000000000000000000ED
:109F30000000000000000000000000000000000021
:109F40000000000000000000000000000000000011
:109F50000000000000000000000000000000000001
:109F600000000000000000000000000000000000F1
:109F7000000000000000000000007E000001FF80E3
:109F8000000380C0000600600004002000040020E0
:109F900000040020020400400202008003FFFFE0F2
:109FA00007FFFFC00000004000000040000000006C
:109FB00000000000000000000000000000000000A1
:109FC0000000000000000000000000000000000091
:109FD0000000000000000000000000000000000081
:109FE0000000000000000000000000000000000071
:109FF000000000000000000000007E000001FF8063
:10A00000000311C000021040000410600004102082
:10A01000000410200004102000061020000310404F
:10A020000001F0C00000710000000000000000000E
:10A030000000000000000000000000000000000020
:10A040000000000000000000000000000000000010
:10A050000000000000000000000000000000000000
:10A0600000000000000000000000000000000000F0
:10A0700000000000000000000004000000040020B8
:10A080000004002000040020007FFFE001FFFFE04B
:10A090000104002003040020020400200204002028
:10A0A000020400000200000001C0000001C0000026
:10A0B00000000000000000000000000000000000A0
:10A0C0000000000000000000000000000000000090
:10A0D0000000000000000000000000000000000080
:10A0E0000000000000000000000000000000000070
:10A0F00000000000000000000000001C0000E33E23
:10A100000003FFC200020CC3000404C1000404C128
:10A11000000404C1000404C100060CC10003F8C31C
:10A120000005F0620006007E0006003C0000000012
:10A13000000000000000000000000000000000001F
:10A14000000000000000000000000000000000000F
:10A1500000000000000000000000000000000000FF
:10A1600000000000000000000000000000000000EF
:10A1700000000000020000200200002003FFFFE0BA
:10A1800007FFFFE0000100200002002000060000A1
:10A19000000400000004000000040020000600206D
:10A1A0000003FFE00001FFE00000002000000020AD
:10A1B000000000000000000000000000000000009F
:10A1C000000000000000000000000000000000008F
:10A1D000000000000000000000000000000000007F
:10A1E000000000000000000000000000000000006F
:10A1F000000000000000000000000000000400203B
:10A200000004002000040020000400200387FFE079
:10A21000038FFFE0038000200000002000000020EA
:10A22000000000200000000000000000000000000E
:10A23000000000000000000000000000000000001E
:10A24000000000000000000000000000000000000E
:10A2500000000000000000000000000000000000FE
:10A2600000000000000000000000000000000000EE
:10A2700000000000000000000000000000000006D8
:10A2800000000007000000010000000100040001C0
:10A290000004000100040003000400060387FFFC23
:10A2A000038FFFF8038000000000000000000000A2
:10A2B000000000000000000000000000000000009E
:10A2C000000000000000000000000000000000008E
:10A2D000000000000000000000000000000000007E
:10A2E000000000000000000000000000000000006E
:10A2F00000000000020000200200002003FFFFE039
:10A3000007FFFFE0000008200000102000003000E0
:10A310000000FC0000058E00000707A0000601E019
:10A32000000400E000040020000000200000000005
:10A33000000000000000000000000000000000001D
:10A34000000000000000000000000000000000000D
:10A3500000000000000000000000000000000000FD
:10A3600000000000000000000000000000000000ED
:10A3700000000000000000000000000002000020BB
:10A3800002000020020000200200002003FFFFE086
:10A3900007FFFFE000000020000000200000002078
:10A3A000000000200000000000000000000000008D
:10A3B000000000000000000000000000000000009D
:10A3C000000000000000000000000000000000008D
:10A3D000000000000000000000000000000000007D
:10A3E000000000000000000000000000000000006D
:10A3F00000000000000400200007FFE0000FFFE065
:10A400000002002000040000000400200007FFE01C
:10A410000003FFE000020020000400000004002010
:10A420000007FFE00003FFE0000000200000000044
:10A43000000000000000000000000000000000001C
:10A44000000000000000000000000000000000000C
:10A4500000000000000000000000000000000000FC
:10A4600000000000000000000000000000000000EC
:10A470000000000000040020000400200007FFE0AE
:10A48000000FFFE000010020000200200002000099
:10A49000000400000004000000040020000600206A
:10A4A0000003FFE00001FFE00000002000000020AA
:10A4B000000000000000000000000000000000009C
:10A4C000000000000000000000000000000000008C
:10A4D000000000000000000000000000000000007C
:10A4E000000000000000000000000000000000006C
:10A4F000000000000000000000007E000000FF805F
:10A50000000381C00002004000060020000400207B
:10A51000000400200004002000060020000200408B
:10A52000000381C00001FF8000007E0000000000E9
:10A53000000000000000000000000000000000001B
:10A54000000000000000000000000000000000000B
:10A5500000000000000000000000000000000000FB
:10A5600000000000000000000000000000000000EB
:10A570000000000000040001000400010007FFFFCC
:10A58000000FFFFF000100C1000200410004002095
:10A590000004002000040020000400200006004009
:10A5A000000301C00001FF8000007E0000000000E9
:10A5B000000000000000000000000000000000009B
:10A5C000000000000000000000000000000000008B
:10A5D000000000000000000000000000000000007B
:10A5E000000000000000000000000000000000006B
:10A5F000000000000000000000007E000001FF805D
:10A60000000380C00002006000040020000400205D
:10A61000000400200004002000020041000300C1EB
:10A620000003FFFF0007FFFF000000010000000122
:10A63000000000000000000000000000000000001A
:10A64000000000000000000000000000000000000A
:10A6500000000000000000000000000000000000FA
:10A6600000000000000000000000000000000000EA
:10A67000000000000004002000040020000400206E
:10A6800000040020000FFFE0000FFFE00000C020EA
:10A69000000100200002002000060020000400004D
:10A6A000000400000007000000030000000000009C
:10A6B000000000000000000000000000000000009A
:10A6C000000000000000000000000000000000008A
:10A6D000000000000000000000000000000000007A
:10A6E000000000000000000000000000000000006A
:10A6F0000000000000000000000003E00001C0E0D6
:10A700000003E04000063020000430200004182040
:10A71000000418200004182000040C2000020C6023
:10A72000000307C000078380000000000000000055
:10A730000000000000000000000000000000000019
:10A740000000000000000000000000000000000009
:10A7500000000000000000000000000000000000F9
:10A7600000000000000000000000000000000000E9
:10A7700000000000000000000004000000040000D1
:10A7800000040000000C0000001FFF8000FFFFC05D
:10A7900000040060000400200004002000040020E9
:10A7A00000040040000001800000000000000000E4
:10A7B0000000000000000000000000000000000099
:10A7C0000000000000000000000000000000000089
:10A7D0000000000000000000000000000000000079
:10A7E0000000000000000000000000000000000069
:10A7F0000000000000040000000400000007FF80CB
:10A80000000FFFC0000000600000002000000020DA
:10A810000000002000000020000400400004008030
:10A820000007FFE0000FFFC00000004000000040F4
:10A830000000000000000000000000000000000018
:10A840000000000000000000000000000000000008
:10A8500000000000000000000000000000000000F8
:10A8600000000000000000000000000000000000E8
:10A870000000000000040000000400000007800049
:10A880000007F0000004FE0000041FC0000003E009
:10A890000000038000001C0000046000000780002E
:10A8A000000600000004000000000000000000009E
:10A8B0000000000000000000000000000000000098
:10A8C0000000000000000000000000000000000088
:10A8D0000000000000000000000000000000000078
:10A8E0000000000000000000000000000000000068
:10A8F00000040000000600000007C0000007FC0084
:10A9000000043F80000003E000040F800006F00018
:10A910000007F0000007FF8000040FE00000038044
:10A9200000043C000007C000000600000004000016
:10A930000000000000000000000000000000000017
:10A940000000000000000000000000000000000007
:10A9500000000000000000000000000000000000F7
:10A9600000000000000000000000000000000000E7
:10A97000000000000000002000040020000400602F
:10A98000000700E0000783200007E6000004F8004D
:10A9900000003C0000045E20000587A0000601E0E6
:10A9A00000040060000400200000002000000000FF
:10A9B0000000000000000000000000000000000097
:10A9C0000000000000000000000000000000000087
:10A9D0000000000000000000000000000000000077
:10A9E0000000000000000000000000000000000067
:10A9F0000000000000040000000400030007000342
:10AA00000007E0010004F80100041F02000007FC39
:10AA1000000000E000000700000438000007C0004C
:10AA20000006000000040000000400000000000018
:10AA30000000000000000000000000000000000016
:10AA40000000000000000000000000000000000006
:10AA500000000000000000000000000000000000F6
:10AA600000000000000000000000000000000000E6
:10AA7000000000000000000000078060000600E009
:10AA8000000403E0000407A000040E2000043C20A2
:10AA9000000470200005E02000078020000700600F
:10AAA000000400E00000038000000000000000003F
:10AAB0000000000000000000000000000000000096
:10AAC0000000000000000000000000000000000086
:10AAD0000000000000000000000000000000000076
:10AAE0000000000000000000000000000000000066
:10AAF0000000000000000000000000000000000056
:10AB000000000000000000000000000000008000C5
:10AB1000000080000001400007FE3FF8080000042C
:10AB20001000000210000002000000000000000001
:10AB30000000000000000000000000000000000015
:10AB40000000000000000000000000000000000005
:10AB500000000000000000000000000000000000F5
:10AB600000000000000000000000000000000000E5
:10AB700000000000000000000000000000000000D5
:10AB800000000000000000000000000000000000C5
:10AB9000FFFFFFFF000000000000000000000000B9
:10ABA00000000000000000000000000000000000A5
:10ABB0000000000000000000000000000000000095
:10ABC0000000000000000000000000000000000085
:10ABD0000000000000000000000000000000000075
:10ABE0000000000000000000000000000000000065
:10ABF0000000000000000000100000021000000231
:10AC00000800000407FE3FF800014000000080003B
:10AC100000008000000000000000000000000000B4
:10AC20000000000000000000000000000000000024
:10AC30000000000000000000000000000000000014
:10AC40000000000000000000000000000000000004
:10AC500000000000000000000000000000000000F4
:10AC600000000000000000000000000000000000E4
:10AC7000000000001800000030000000400000004C
:10AC800040000000400000002000000030000000F4
:10AC900008000000040000000200000002000000A4
:10ACA000020000000C00000018000000000000007E
:10ACB0000000000000000000000000000000000094
:10ACC0000000000000000000000000000000000084
:10ACD0000000000000000000000000000000000074
:10ACE0000000000000000000000000000000000064
:10ACF00030313233343536373839414243444546B2
:10AD000040305800303132333435363738396162AB
:08AD10006364656640307800C1
:040000050800029954
:00000001FF
